:020000040800F2
:10000000F81E0020A5860008E5860008B31F00083A
:10001000E9860008EB860008ED8600080000000075
:10002000000000000000000000000000EF86000853
:10003000F186000800000000F386000889680008C7
:10004000F7860008F7860008F7860008F78600089C
:10005000F7860008F7860008F7860008F3710008A5
:10006000F7860008F7860008F7860008F78600087C
:10007000F7860008F7860008A76A0008F7860008D8
:10008000F7860008F7860008F7860008F78600085C
:10009000F7860008F7860008F7860008F571000863
:1000A000F7860008F7860008F7860008C364000892
:1000B000AF650008B7650008BD6500085760000817
:1000C000355E00085B60000859600008F78600088C
:1000D000F7860008F78600085D6D0008F7860008BF
:1000E00049590008F7860008F7860008DFF80CD0A9
:1000F00009F07EF9004800473F1E0008F81E002066
:1001000070B51546B0FBF5F60446A84203D3304659
:10011000FFF7F6FF014605FB1640FAA2105C0870D7
:10012000481C70BD70B50C46911E232900D30A22CD
:100130000025002804DA2D212170611C404200E0D6
:100140002146FFF7DDFF0570204670BD2DE9F05F09
:10015000044600E0641C2278202AFBD0092AF9D04A
:10016000DFF8C8A3D0B24FF000092D2802D02B2A07
:1001700004D004E0DFF8B8A34FF00009641C0026A7
:100180003746DFF8B0B310E008F012FF05468846A6
:1001900000225B463046394608F01DFE43462A469B
:1001A00008F073FD06460F46641C20783038092895
:1001B000EAD920782E281CD10025DFF8788313E0B7
:1001C00008F0F6FE2A46434608F075FE32463B46E6
:1001D00008F05BFD06460F4600225B462846414676
:1001E00008F0F9FD0546884614F8010F3038092853
:1001F000E6D922780020CD49652A01D0452A42D18E
:1002000014F8012F4FF000082D2A02D02B2A02D01B
:1002100002E04FF00108641C00256FF02F0C05E090
:1002200005EB85030CEB4303D518641C2278A2F17F
:100230003003092BF4D94FF49A72954205D915462B
:10024000BD4ABE4B08F0C7FD323D322DF8D2BC4C42
:10025000082D0BD30022234608F0BDFD083DF7E72B
:100260000022234608F0B7FD6D1E00E05C46002D1D
:10027000F6D1B8F1000F06D002460B46304639469B
:1002800008F019FE03E032463B4608F0A4FD4A465A
:10029000534608F0A0FDBDE8F05F08F0FCBEF0B5E5
:1002A00087B000260D46A84900960196A5A702969C
:1002B000B0F5000F02DB08F00EFC01E008F05DFC79
:1002C000A24908F060FC08F084FE041E00DC6042D5
:1002D0000A2203A9FFF726FF002C01DB202000E003
:1002E0002D208DF8000003A808F0C7FB302401285A
:1002F0000AD003A808F0C1FB02280CD003A808F01C
:10030000BCFB03280CD00DE08DF801408DF80240B5
:100310008DF8034006E08DF801408DF8024001E0C1
:100320008DF8014003A9684608F06EFB684608F0A6
:10033000A4FBC01EC4B222466946284608F088FBCA
:100340002E553946284608F05FFB0DEB0401284680
:1003500008F05AFB07B02846F0BD70B505460C46BC
:10036000086808F08AFB024621682868BDE87040EA
:1003700008F08BBB2DE9F041002488B007462646E3
:1003800008F07BFB724D10F0FF0F4ED0042271A1DC
:10039000384608F07AFB00287DD0384608F08EFBFE
:1003A000461E0C2E78DA2021384608F05DFB070047
:1003B00008D0471C3846FFF7C9FE05EB061101249B
:1003C000C1F8FC002021384608F04EFB070008D099
:1003D000471C3846FFF7BAFE05EB0611641CC1F84E
:1003E00000012021384608F03FFB070008D0471CD9
:1003F0003846FFF7ABFE05EB0611641CC1F804019B
:100400002021384608F030FB38B1401CFFF79EFE33
:1004100005EB0611641CC1F80801042C70D04FA034
:1004200006F00EFC08B0BDE8F0815BA006F008FC09
:1004300000240DF1100800BF05EB0417D7F8FC00ED
:1004400010F0FF4F2ED0002148F82410761C611CBC
:100450005CA008F074FA57F8FC0F6946FFF71FFF1D
:1004600001465AA008F06BFA69467868FFF717FF53
:10047000014656A008F063FA6946B868FFF70FFF17
:10048000014652A008F05BFA6946F868FFF707FFDB
:1004900001464FA001E0ADE0D3E008F050FA641C43
:1004A0000C2CC9DB002413E005EB041707F580775B
:1004B0000498396808F00FFB04907968059808F0F3
:1004C0000AFB0590B968069808F005FB641C0690C5
:1004D000B442E9DB40A006F0B3FB434E002445469E
:1004E00055F8240020F00040B04201DD3FA000E0BC
:1004F0003FA006F0A5FB641C032CF1DB30A08FE7C6
:100500009AE00000303132333435363738394142E1
:10051000434445464748494A4B4C4D4E4F50515233
:10052000535455565758595A000000000000F03FE8
:100530000000F0BF000024409A647EC50E1B514AA3
:1005400084D797412E0000006F12033A00007A44CE
:10055000040500206C6F61640000000057726F6E2C
:1005600067206E756D626572206F662061726775B7
:100570006D656E74732C206E656564732069647894
:100580002074687220726F6C6C20706974636820CC
:100590007961770D0A000000437573746F6D206DEB
:1005A000697865723A200D0A4D6F746F720954684C
:1005B0007209526F6C6C09506974636809596177EC
:1005C0000D0A00002325643A090000002573090084
:1005D00025730D0A0000000053616E697479206371
:1005E0006865636B3A0900000AD7233C4E4709004F
:1005F0004F4B09002021384608F036FA00283FF416
:1006000011AF401C054608F038FAF14EC7B200247D
:1006100056F8241031B13A46284608F036FA18B197
:10062000641CF5E7EBA0FBE6204601F02CFD56F834
:100630002410EEA008F083F9AFF21410FFF79AFE31
:10064000F0E60C21EEA008F07AF9EBE610B5F6A082
:1006500006F0F6FA012000F0C3FEFAA006F0F0FA68
:100660000A2006F039F9BDE81040002006F0DCB998
:1006700010B5F8A006F0E4FA002000F066FDF8A03E
:1006800006F0DEFA0A2006F027F9BDE81040002047
:1006900006F0CAB910B50446F5A006F0D1FA30212B
:1006A000F94808F0A5F9CA480021001F0160F74881
:1006B00001702046BDE81040DAE72DE9F047064614
:1006C00008F0DBF9054600F0E9FEDFF80493074681
:1006D0004FF0010809F14C0955B12A46ECA130460A
:1006E00008F0D3F9C0B1307800272D2823D025E0B9
:1006F000E9A006F0A5FA002445464E4656F8241017
:1007000041B105FA04F0384202D0E8A008F017F928
:10071000641CF3E7B9A01EE0E5A006F091FA0024FE
:100720004FEA090555F824100029F3D0DFA008F09E
:1007300006F9641CF6E70127761C6D1E5FF00004C5
:1007400059F8241031B12A46304608F09EF930B1EC
:10075000641CF5E7DCA0BDE8F04706F071BA08FAC2
:1007600004F01FB100F095FEDEA002E000F02FFDC6
:10077000DFA006F065FA59F82410AFF2AC10BDE81E
:10078000F04708F0DCB870B50024DCA006F058FA99
:10079000E04D00BF04EB440005EB80014A6855F8CA
:1007A0002010DDA008F0CBF8641C0B2CF2D370BD38
:1007B0003EB5054608F061F908281DD10024285DE2
:1007C00008F0D4F82855641C082CF8D30024D44829
:1007D000295D08F049F928B12819295D401C08F065
:1007E00043F918B1CFA006F02BFA3EBD641C082CCB
:1007F000EDD3284600F022FCD2A006F021FAC84B27
:10080000D64A0020694615181C5C95F88150401C9A
:1008100008284C55F7D300220A54AFF24C2008F0B8
:100820008EF83EBD2DE9F041804608F026F9CB4F09
:10083000674D10F0FF0612D0324695A1404608F0F1
:1008400024F998B15FF0000455F82410E9B132465C
:10085000404608F01AF9E8B1641CE4B2F4E778798C
:1008600005EB800050F8041CBDA018E0C1A006F004
:10087000E7F9002455F8241029B18CA008F05FF89E
:10088000641CE4B2F6E75DA000E052A0BDE8F041D0
:1008900006F0D6B9601C787155F82410BAA0BDE8EE
:1008A000F04108F04CB87CB504460D4600790021B3
:1008B000062814D2DFE800F003060A0D111EA06816
:1008C00001780CE0A06890F9001008E0A0680188A9
:1008D00005E0A068B0F9001001E0A0680168AFA0D1
:1008E00008F02DF8002D04D0D4E90312ACA008F0D4
:1008F00026F87CBDA06869460068FFF7D0FC014679
:10090000A9A008F01CF8002DF3D0E06808F042FB25
:100910006946FFF7C4FC0146A4A008F010F820695E
:1009200008F038FB6946FFF7BAFC01469FA008F0C3
:1009300006F87CBD2DE9F047814608F09EF8754C1D
:10094000060004F1840429D0012E03D199F8000097
:100950002A2823D096A1484608F064F8002834D00D
:10096000401C054608F0AAF882462846FFF7EEFB31
:100970008046002606EB860704EB870554F827001F
:1009800008F07BF8024654F82710484608F07DF836
:10099000E8B1761C552EEDD386A05DE18DA006F062
:1009A0004FF9002505EB850004EB800754F8201073
:1009B0008EA007F0C4FF31463846FFF774FF0FA042
:1009C00006F03EF96D1C552DECD3BDE8F08711E122
:1009D00004000020496E76616C6964206D69786559
:1009E0007220747970652E2E2E0D0A004C6F616492
:1009F0006564202573206D69782E2E2E0D0A000067
:100A00004D6F746F72206E756D626572206D7573B7
:100A100074206265206265747765656E203120619F
:100A20006E642025640D0A00526573657474696EE6
:100A30006720746F2064656661756C74732E2E2E4A
:100A40000D0A00005265626F6F74696E672E2E2E5C
:100A500000000000536176696E672E2E2E000000A4
:100A60000D0A5265626F6F74696E672E2E2E00003C
:100A70000D0A4C656176696E6720434C49206D6FA5
:100A800064652E2E2E0D0A00D40400204902002099
:100A90006C69737400000000456E61626C656420CF
:100AA00066656174757265733A20000025732000D5
:100AB000417661696C61626C65206665617475720E
:100AC00065733A2000000000496E76616C6964200D
:100AD00066656174757265206E616D652E2E2E0DD2
:100AE0000A00000044697361626C656420000000C4
:100AF000456E61626C6564200000000041766169AA
:100B00006C61626C6520636F6D6D616E64733A0D2C
:100B10000A0000005CA9000825730925730D0A006E
:100B200084B000084D75737420626520616E792071
:100B30006F72646572206F662041455452313233C2
:100B4000340D0A0043757272656E742061737369A7
:100B5000676E6D656E743A20000000000405002089
:100B600043757272656E74206D697865723A2025DE
:100B7000730D0A00417661696C61626C65206D6974
:100B8000786572733A2000004D697865722073654C
:100B90007420746F2025730D0A0000002564000086
:100BA00020256420256400002573000020257300A3
:100BB0003D0000004552523A20556E6B6E6F776EC5
:100BC000207661726961626C65206E616D650D0AE7
:100BD0000000000043757272656E74207365747452
:100BE000696E67733A200D0A000000002573203DEE
:100BF0002000000006EB860704EB8706F06808F08B
:100C0000C9F9414608F064FA25D8306908F0C2F9FC
:100C1000414608F067FA1ED83179052907D05046B9
:100C200006290ED2DFE801F0050508080B0B404647
:100C3000F6E7A968087004E0A968088001E0A968DF
:100C4000086054F8271096A007F079FE2846BDE802
:100C5000F047002127E695A0BDE8F04705F0F0BF7A
:100C60002DE9F04105F02AFE4FF47A71B0FBF1F165
:100C7000984803789848027898A007F060FE00F042
:100C8000FDFB0646A548A6490068B0FBF1F1A5A00A
:100C900007F055FE0024AB4F012500BF57F8241084
:100CA00051B105FA04F0304203D0AFF2002007F052
:100CB00046FE641CE4B2F1E7012000F0CDFB40B138
:100CC000A149A0480978183050F821109FA007F0DA
:100CD00036FEAFF2D82005F0B3FF05F047FA024622
:100CE0009D480188BDE8F0419CA007F028BEA4A063
:100CF00005F0A6BF2DE9FF5FDFF8B49299F8000078
:100D000038B9012189F80010AAA005F099FF00F078
:100D1000C4F8DFF830A2DFF8D4B2AAF1840A00BF29
:100D200005F05EFF00286ED005F070FF092806D0A0
:100D30003F2804D0DAF800105446B1B34DE0AC4F70
:100D40000024254607F18408DAF800600CE000BFB3
:100D5000DAF8002022B1A548396807F096FE10B9EC
:100D600004B93C463D460C374745F1D39CB150464B
:100D70005F46016822682B68525C5B5C9A420AD12C
:100D80001AB17A54491C0160F3E720220BF80120C4
:100D9000491CCAF80010DAF80000574608B1AC4206
:100DA00010D094A005F04CFF07E014E0206805F097
:100DB00047FF092005F037FF0C34AC42F6D900F0AC
:100DC0006CF800265C4638688642A9D2A05D05F022
:100DD0002AFF761CF7E7042810D00C2814D019B18C
:100DE0000A2815D00D2813D07F283ED0302997D25D
:100DF000202895D37E2893D8B1B344E004B07B4833
:100E0000BDE8F05F46E446E07CA005F019FF28E06D
:100E1000AFF2184005F014FF206800255E460BF87D
:100E200000507948CDE9000B0C230B227049029544
:100E300001A807F0A1FD070007D0386807F01DFEE4
:100E40003044B968401C884702E070A005F0F8FE05
:100E50003021664807F0CCFD256099F80000002895
:100E600019D000F01AF85BE70BE00029FBD0491E0F
:100E70000020CAF800100BF801006DA005F0E0FE9C
:100E80004EE72028EFD00BF80100491CCAF80010EB
:100E900005F0C9FE44E7BDE8FF9F66A005F0D0BE9F
:100EA00025732073657420746F2000004552523AF8
:100EB0002056616C75652061737369676E6D656E30
:100EC00074206F7574206F662072616E67650D0AFD
:100ED00000000000F30100204401002053797374E6
:100EE000656D20557074696D653A202564207365C1
:100EF000636F6E64732C20566F6C746167653A2063
:100F00002564202A20302E31562028256453206263
:100F1000617474657279290D0A000000A004002034
:100F200040420F004350552025644D487A2C2064E0
:100F3000657465637465642073656E736F72733A6C
:100F40002000000084000020FC01002041434348B1
:100F5000573A202573000000460100204379636C56
:100F6000652054696D653A2025642C204932432060
:100F70004572726F72733A2025640D0A00000000FA
:100F80004166726F333220434C4920766572736933
:100F90006F6E20322E31204F637420203620323085
:100FA0003132202F2032333A33313A3034000000CE
:100FB000490200200D0A456E746572696E67204310
:100FC0004C49204D6F64652C20747970652027652D
:100FD0007869742720746F2072657475726E2C2086
:100FE0006F72202768656C70270D0A00D4040020FA
:100FF0005CA900080D1B5B4B000000001B5B324A24
:101000001B5B313B314800005B0300084552523AFC
:1010100020556E6B6E6F776E20636F6D6D616E64C1
:101020002C20747279202768656C702700000000FE
:10103000082008000D0A2320000000002DE9F041DF
:1010400005460446F74EF84F09E0F64807F00CFD58
:1010500020B1611B801B384480F88110641C21780A
:101060000029F2D1BDE8F0812DE9F05F4FF4E07284
:10107000EE49ED4807F0A3FCEB48ED4E002190F857
:101080002D2090F82C4040F6C41500BF01FB01F361
:10109000193B534303F6C4134B43634393FBF5F3EC
:1010A00026F81130491CC9B20629EFD390F82F2039
:1010B000B0F89A409246C2F1640C90F82E30B0F825
:1010C0009C200021DFF86CB34FF00A0E03EB83087D
:1010D000A146151B01EB8102C3EB42040122002C47
:1010E00003DDC3F16402D2B201E000DA1A4604FB68
:1010F00004F70AFB07F602FB02F296FBF2F26244E7
:1011000002FB04F292FBFEF202EB480212B205FB74
:1011100002F24FF47A7492FBF4F404EB09022BF818
:10112000112001F10101C9B20B29D3D3B0F8BE10CF
:10113000B0F8C020914203D3B0F8C220914200D948
:101140001146A0F8BE10BDE8F09F2DE9F041BA4964
:10115000B54C4FF4E0760978217080466680BE2158
:1011600000202171EF2184F8BC11214684F8BD01D3
:1011700001F5E07203E000BF11F8013B58409142D5
:10118000FAD384F8BD0107F019FA342007F080FA89
:10119000A64F384607F040FA042809D10025E8197F
:1011A000615907F055FA042802D12D1DB542F6D336
:1011B00007F00AFAFFF758FFB8F1000F06D0BDE8B4
:1011C000F041012214210F2001F0D6B94AE79649D7
:1011D0008A6802438A6070472DE9F05F4FF4E0713E
:1011E000914807F005FC94488F4C0025007820704A
:1011F000032060710220A560FFF7E9FFA581282187
:10120000A1734FF01E0B84F818B010341722A2748B
:1012100004F8011C84F809B0E274552020702D22D6
:10122000A2722575102060700F20E0720720607593
:101230000B20A0702573A5754FF0140884F8038067
:1012400008236373E2750E22227184F80E80502207
:101250002276462262710A27E77384F81980A17109
:10126000E5716574E5765A2020774120607784F82F
:10127000205084F8215084F822503220A077E5775E
:10128000A4F110044FF0000104EB410201F101014F
:10129000A2F860500F29F7DB04F134044FF0040189
:1012A000E581258225806580A580A581A574E174EE
:1012B00004F8147F814660704FF4C87AA4F804A043
:1012C0004FF02A0060804FF0010626734FF01500A2
:1012D00060735A4820615A4860615A48A0604FF0D4
:1012E0006E0084F836004FF02B0084F837004FF082
:1012F000210084F8380004F1700453A0FFF79EFE2B
:1013000004F82F5C04F82E5C04F82D8C04F82C5D96
:1013100040F2DC50608040F24C41A18004F12C048A
:1013200040F26C7124F8261C04F8245DC4466770F2
:101330004FF0C80884F802804FF49661A18040F213
:101340007E41E18040F23A71218104F124044FF49E
:101350007A7124F81A1C24F818AC24F8169C26710B
:10136000E0804FF47F7121814FF4FA626281A181A4
:10137000E08122826182A082E28226764FF0FF0322
:101380006376A676E67627776777A67721846284E8
:10139000A084E1842285608584F82C504FF4E130EC
:1013A0002063A4F8348084F836C084F837B084F819
:1013B00038604FF0640161874FF49671A187206413
:1013C000A4F1B8044FF0000004EB001100F101009B
:1013D000C1F8FC500C28F7DBBDE8F05F0020B4E654
:1013E00030B41249144C00220B7825781446AB42D5
:1013F00013D14B88B3F5E07F0FD10B79BE2B0CD105
:1014000091F8BC31EF2B08D101F5E07311F8015BC5
:101410006A409942FAD302B90124401E044219D10C
:1014200030BCD9E684B000080405002000FC0108A7
:101430009C080020A8080020B00000209A99193FBD
:10144000F6287C3F031414004145545231323334A2
:101450000000000030BC704712494968014201D0C9
:1014600001207047002070470E494A6802434A60D5
:1014700070470C494A6882434A607047094840688F
:10148000704709498968014201D001207047002056
:10149000704705498A6882438A60704702488068BD
:1014A00070470000B00000200405002070B5FE4821
:1014B000008807F078FD0446FC4907F064FB07F05C
:1014C00088FDFB4D21466880FA4807F092FBFA49F7
:1014D00007F08FFBE8630420FFF7BEFF002803D06E
:1014E000BDE8704002F032BA70BD2DE9F04F91B006
:1014F000D0E900458046866848680F4680F0004085
:1015000008F074FB8246786880F0004009F024F906
:101510008346386808F06AFB0190386809F01CF9C6
:101520008146B86808F062FB0490B86809F014F9C5
:1015300005905146049807F026FB069001990498FF
:1015400007F021FB07465146059807F01CFB079062
:101550005846049907F017FB04905846059907F080
:1015600012FB08900199059807F00DFB059089F092
:1015700000400C904946049807F005FB079907F0D6
:10158000FCFA0D904946089807F0FDFA069907F015
:10159000A2FA0E905946019807F0F5FA03904946D1
:1015A000069807F0F0FA089907F095FA834649463D
:1015B000079807F0E8FA049907F0DFFA009051461F
:1015C000019807F0E0FA01903046594607F0DBFA3F
:1015D000824628460D9907F0D6FA814639462046BC
:1015E00007F0D1FA494607F076FA514607F073FA48
:1015F000C8F800003046009907F0C5FA8146284631
:101600000E9907F0C0FA07462046059907F0BBFA85
:10161000394607F060FA494607F05DFAC8F8040059
:101620003046019907F0AFFA06462846039907F0BD
:10163000AAFA054620460C9907F0A5FA294607F0B4
:101640004AFA314607F047FAC8F8080011B0BDE879
:10165000F08F2DE9F04F89B0002605F01AF9944C6F
:101660000546E069281A07F09EFC944907F08BFABA
:101670000290DFF83CA2E5610AF1580A904D00247F
:101680004FF07E580AF106098948523030F91400AB
:1016900007F080FC029907F076FA06A941F82400C9
:1016A00095F8470010B307F07EFC014647464046D8
:1016B00007F09FFA04903AF9140007F06BFC0499C4
:1016C00007F061FA83463946049807F059FA7D4FCE
:1016D00057F8241007F057FA594607F0FCF947F875
:1016E000240007F076FC29F8140003E03AF81410FF
:1016F00029F8141095F8480007F055FC01464746B4
:10170000404607F076FA83463AF9140007F042FCA7
:10171000594607F038FA03903946584607F030FA30
:10172000684F6C3757F8241007F02DFA039907F02B
:10173000D2F947F8240039F9140000FB00660420B0
:10174000FFF78AFE641C032C9ED364204643564850
:1017500006A90088404396FBF0F407F10C00FFF760
:10176000C4FE0420FFF778FE20B106A9A7F1780097
:10177000FFF7BBFEB9F900004F46002800DC4042ED
:10178000DFF82C915049B9F9022090420CDAB7F9F0
:101790000200002800DC4042904205DAB7F904005C
:1017A000002801DD012000E00020464E253C78366F
:1017B00048739F2C02D310F0FF0F22D00024B5F8FD
:1017C0004C0007F0F0FB8246414607F084F90146E1
:1017D000404607F00EFA804637F9140007F0DAFBAE
:1017E000054656F82410504607F0CDF9294607F073
:1017F00072F9414607F0C7F946F82400641C032C2F
:10180000EAD30420FFF728FE2E4C0C3CE8B1DFF8A9
:10181000A080DFF8B8A0DFF8B8B0002508F16408B0
:1018200038F9150007F0B6FB074654F82500514675
:1018300007F0A9F9394607F04EF9594607F0A3F920
:1018400044F825006D1C032DEAD3B168306800F020
:10185000E1FA174D14352880B068014607F093F976
:1018600080467068014607F08EF9074630680146E9
:1018700007F089F9394607F02EF9414607F02BF9B0
:1018800009F056F880F00041706807F0B2F907F0EF
:10189000EFFF104907F077F907F09BFB6880042001
:1018A000FFF7DAFD002817E0040200207593D83E08
:1018B000B80000200AE81C4100401C465344923105
:1018C00004050020D00600208C08002000004843BA
:1018D0005E06A33B4C3D0FC437D0A568706829460F
:1018E00007F051F9B76880466168384607F04BF950
:1018F000414607F042F980463846216807F043F92F
:1019000004462946306807F03EF9214607F035F9CC
:10191000414600F07FFAFE4C07F03CFBD9F810106E
:1019200007F0D9F807F055FB00B20A2190FBF1F05F
:1019300000B22080B42802DDA0F5B47004E010F1FC
:10194000B40F02DA00F5B470208009B07FE62DE90B
:10195000FF5F0120FFF780FD18B101F00AFFFFF7DC
:1019600078FE01F0D6FFEB4C00256F46AA4604F145
:10197000060B00BF34F8150027F815000120FFF70B
:101980006BFD08B92BF815A06D1C032DF2D304F0E4
:1019900080FFE04E523EB06100F018FE04F079FF87
:1019A000B16940F28A25401AA84204D9DA48018870
:1019B000491C018005E004F06CFFB169401AA8429F
:1019C000F9D301F0A6FFA046B946D24C0025032763
:1019D000B4F1120438F8151039F81500084402A9BA
:1019E00000B221F81500CB490C3931F91520024419
:1019F00092FBF7F200EBD07024F81520401021F88C
:101A000015000120FFF728FD08B92BF815A06D1C63
:101A1000032DDFD34020FFF734FDC04A00B3BD499A
:101A20004839087828B9106D020C0A70020A4A7009
:101A30008870B84D0020AD1F0A5C34F9106035F98C
:101A40001070531E07FB03635B1C93FBF2F224F838
:101A5000102025F81020401C0328EDD3BDE8FF9F7F
:101A600050790128FAD1B4F90400B6F9081000EB56
:101A7000410090FBF7F0A0803081EFE7002801DD06
:101A8000024600E042428A4201DA00207047002804
:101A900002DDA0EB010001E0F8DA084400B2704773
:101AA00070B50446084607F075FA05464FF400067F
:101AB0002946B44201DB204601E084F0004007F0F3
:101AC00007FB01D200240EE0B44204DB2146284685
:101AD00007F056F806E014F1FF4F04D321462846DC
:101AE00006F0F9FF0446204670BD70B58C49A1EBA5
:101AF0006004214607F047F8214607F044F8894979
:101B000007F03EF805464FF0FF31204607F0B1F8E8
:101B10002946BDE8704007F036B82DE9FC5F8248E1
:101B20007C4C46F2A812523C0168206A081A904286
:101B30007EDB21628146216B0A2091FBF0F001B22D
:101B40007A4D94F9000025F81010626A401C0A448E
:101B5000724991F8556090FBF6F306FB130340B20F
:101B600035F91330D51A65622070864201D1002004
:101B700020708F6D884639464FF07E5006F0FDFF8D
:101B80008246701E07F006FA0646284607F002FA5B
:101B9000674906F0F8FF314607F02BF8514606F08A
:101BA000F2FF0546606B07F0F5F9394606F0EBFFEA
:101BB000294606F090FF07F00CFA6063A16B081A43
:101BC0005C49884202DB4942884200DD084600B297
:101BD0000A21FFF753FF98F811306421434393FB28
:101BE000F1F16FF09505A94201DA294604E043F6C8
:101BF000FB25AB4200DD962109B2A18098F81B209D
:101C00004243322092FBF0F2E088104400B24A4A8C
:101C1000E080904202DB5242904200DD1046E080BC
:101C20004FF4FA7290FBF2F00844A0803F4D00E0C0
:101C3000EEE06C35286807F0CCF900FB00F6686828
:101C400007F0C7F900FB0066A86807F0C2F9404337
:101C5000304407F09FF9FFF748FF074637480088F0
:101C6000009007F0A0F90190A5F10C06A968B068F2
:101C700006F089FF83466968706806F084FF824633
:101C80002968306806F07FFF514606F024FF594668
:101C900006F021FF394606F076FF019906F06DFF48
:101CA00007F097F998F84920009900B2B1FBF2F1DA
:101CB000454609B2FFF7E2FE214F06463880484606
:101CC00007F071F98046304607F064F9E16B06F0E1
:101CD0005AFF414606F057FFA16A06F0FCFEA062DB
:101CE0001849404606F085FF0646E16A606B401AD7
:101CF00007F050F9314606F07CFF1349884202D8BC
:101D00001249884200DD08460A21FFF7C9FE1FE09C
:101D1000440200200A010020EC01002004050020FC
:101D2000DF59375F0000404064010020DC060020DE
:101D300000002041D4FEFFFFD08AFFFF04020020F4
:101D4000B201002000247449000096C300009643AD
:101D50008046606BE062404607F03BF97880EE6DAC
:101D60004FF07E50314606F008FF414606F00BFF6B
:101D700080463146A06A06F006FF414606F0ABFEFB
:101D80000646A06207F025F9B88005213046FFF726
:101D900087FE064695F8250007F005F9314606F05E
:101DA000F2FE214E314606F024FF2049884212D827
:101DB0000521A06AFFF774FE804695F8250007F01C
:101DC000F2F8414606F0DFFEB046314606F011FF5C
:101DD0001749884201DD08460EE00521A06AFFF799
:101DE0005FFE064695F8250007F0DDF8314606F05F
:101DF000CAFE414606F0FDFE0546B4F9040007F0B0
:101E0000C9F8294606F0B9FE07F0E3F8A080F8808B
:101E1000BDE8FC9F10B507F0BFFD064906F0B3FE14
:101E200007F0D7F800B210BD0000A041000016C3B3
:101E3000000016434C3D0F44084604F0F4BE0EB5B6
:101E400004F055FD5E49002006F075FD0020FFF707
:101E5000C7FAFFF709F95B4CD4F8F80001F05DFF11
:101E60000720FFF701FB0820FFF70BFB564D4FF44F
:101E7000807620B103F0CFF95448286007E030465F
:101E8000FFF7FFFA18B1D4F8E80003F045F8012095
:101E9000FFF7F7FA30B14FF48060FFF7F2FA08B1BC
:101EA00001F081FE00F0A4F860794FF001080E28DF
:101EB0006DD008286BD000208DF805003046FFF764
:101EC000E0FA8DF802000120FFF7DBFA8DF801003F
:101ED0000820FFF7D6FA80F001008DF800003C489A
:101EE000007800B101208DF8030094F8D600C0F30B
:101EF000C0008DF80400B4F8A000ADF80600B4F8F6
:101F0000A200ADF80800684604F0A4FB324931484D
:101F10004FF0100A2860C1F800A00E1F4FF008090A
:101F2000C6F800900025A6F1040B8F14DBF8001012
:101F300081F01001CBF80010DBF8001081F00801EF
:101F4000CBF80010192004F0C7FC244807601920C2
:101F500004F0C2FC2148001F07606D1CEDB20A2D81
:101F6000E4D3C6F80090C6F800A001F061FAFFF7CC
:101F70009DFA0220FFF785FA08B101F012FB04F088
:101F800088FC174908606079052803D006E08DF8C1
:101F9000058093E713494FF4C870088012494FF445
:101FA0007A700880114981F80D8000BF00F038FD7B
:101FB000FCE70448B0F99E0000F0CFF8FEE700000F
:101FC000391E0008040500206C0100204152000861
:101FD0002B0100203B290008140C0140140801408B
:101FE0006801002000020020020200208C0800206E
:101FF0002DE9F041FE4DFF4EFF4C687906EBC00025
:10200000407860702020FFF73CFA08B10120607032
:102010006879DFF8E8C3122809D016F8301006EB0B
:10202000C00021704268002A1CD0002028E0002057
:1020300005EB0011D1F8FC2012F0FF4F12D001F592
:1020400080710CEB0013D1E90067896800F1010091
:10205000C3E90271C3E9002621780C2801F10101CE
:102060002170E5DBBDE8F08102EB00130CEB0014FE
:1020700093E8E000DB68401CC4E90273C4E9005641
:102080008842F1DBEEE7F0B5401C0021DFF860C3C9
:102090000A4600BF0CEB0113491CC3F8FC200C29B5
:1020A000F8DBD44B03EBC0014A68002A15D00021AD
:1020B00013F830000FE000BF02EB01130CEB01142A
:1020C00093E8E000DB6804F1FC0401F10101C4E9DC
:1020D0000273C4E900568842EEDCF0BDC64810B574
:1020E0004078002827D0C248C34C4079A41C05285A
:1020F0000ED004DC01281BD0042804D112E00828EB
:1021000006D00E2817D02020FFF7BBF9002812D0E8
:102110002188002004F020FB61880120BDE81040E8
:1021200004F01ABB2189002004F016FB6189F4E752
:1021300061890020F2E710BD70B5B04E0024183E52
:10214000AD4D06E036F81410204604F0F9FA641C90
:10215000E4B228788442F5D370BDA74AA74B00218A
:102160001278183B04E000BF23F81100491CC9B2E3
:102170009142F9D3E0E72DE9FF5F9F4FDFF880A29E
:102180003B78032B24D99F48BAF90420B0F9040006
:102190004142002801DD044600E00C466FF0630672
:1021A000341BA24204DA002800DC0846301A0DE095
:1021B000002801DD044600E00C466434A24204DD40
:1021C000002800DC0846643000E01046AAF804004D
:1021D0008748DFF828B2012B90F9BC708948ABF131
:1021E000180BB0F9060000908548B0F90260B0F90C
:1021F000009033D9002498462EE000BFBAF90400BD
:10220000784306F0C7FE7D4901EB0415E96806F046
:10221000BAFC0190484606F0BDFE696806F0B3FCC2
:102220000290304606F0B6FEA96806F0ACFC0390BA
:10223000009806F0AFFE296806F0A5FC039906F0A9
:102240004AFC029906F047FC019906F044FC06F0AE
:10225000C0FE2BF81400641C4445CFD3644C664D7B
:10226000DFF8A4816079AD1C052835D004DC012895
:1022700022D0042862D102E008285FD1E9E0BAF94F
:1022800004304FF47F7107FB036202F2DC524FF41B
:10229000FA608A4201DA0A4602E0824200DD024622
:1022A0002A815F43BA1B02F2DC528A4212DB82426D
:1022B00000DC1046688141E0B4F8BE10BAF90400B1
:1022C00007FB0010B4F8C010884203DBB4F8C2105A
:1022D0008842EFDD0846EDE74C4994F9D400494EB9
:1022E000B1F902205043B4F8DC20B6F902301A44A8
:1022F000C31700EB137002EB2010B4F8D820904203
:1023000003DBB4F8DA20904200DD1046288094F90F
:10231000D500B1F90010B6F900204843B4F8E21036
:102320001144C21700EB127001EB2010B4F8DE105C
:1023300088426FDBB4F8E010CFE068802020FFF720
:10234000A0F8E8B394F8D61000208A0707D0B8F8B0
:102350000C20B4F88E30A2EB030262F30F004907A1
:1023600006D4B8F80E10B4F88E20891A61F31F4015
:10237000B4F8DC1001440AB22A80B4F8E21001EB90
:10238000104001B2224869800079B0B11F4E94F923
:10239000D400B6F902305843C31700EB137002EBB8
:1023A0002010288094F9D500B6F900205043C217B8
:1023B00000EB127001EB20106880B5F9000000E01E
:1023C00015E0B4F8D810884203DBB4F8DA1088427C
:1023D00000DD08462880B5F90200B4F8DE10884216
:1023E00003DBB4F8E010884200DD0846688012E0A4
:1023F0000405002080B400082A0100206C0700209A
:10240000AC010020BA010020DC010020CC0000203B
:10241000BE08002064E094F8D600000712D500261C
:102420002020FFF72EF800B1022600254FEA08070A
:1024300007EB45000189A819C0B204F08DF96D1CA5
:10244000042DF5D349495E46BBF9007001200B7895
:102450004EE00098ABF80000464B454893F9D07029
:10246000817A93F9D22093F9D10093F9D33091B1C5
:10247000B8F90210B4F88E60A1EB060C0CFB07F162
:10248000B8F900700CFB00FCBE1B02FB061103FB3D
:1024900006C0298006E0774302FB0971704303FB05
:1024A000090029806880B5F90000B4F8C610084416
:1024B000B4F8C410884203DBB4F8C810884200DDC9
:1024C00008462880B5F90200B4F8CC100844B4F8E6
:1024D000CA10884204DBB4F8CE1088427FF72DAFD3
:1024E00008462AE736F91020BA4200DD1746401C9C
:1024F0009842F7D30025894632E000BFB4F89C002B
:10250000B84205DA36F815103A1A891A26F8151065
:1025100036F91510B4F89A20914201DA104602E01B
:10252000814200DC084626F81500B8F90600B4F828
:102530009010884208DA1020FEF7A3FF40B1B4F8EB
:102540009E0000BF26F815000948407818B106E043
:10255000B4F89A00F6E7B4F89E0026F815006D1C52
:1025600099F800008542C9D3BDE8FF9F2A010020E9
:102570008C080020040500202DE9F74FDFF848A45F
:10258000074690460025DFF83C944FF48056AAF1A8
:10259000040B17E000240EE0D9F8001081F00801C8
:1025A000C9F80010CAF80060019804F095F9CBF85A
:1025B0000060641CE4B2BC42EED33C2004F08CF911
:1025C0006D1CEDB24545E5D3BDE8FE8F2DE9FC5FFE
:1025D000FE4B002440F2DC50B3F90610FC4E4FF4E1
:1025E000FA75814201DA64200DE0F948B1F5FA6F1D
:1025F00090F8320004DAA1F2DC52504390FBF5F07F
:10260000C0F16400C0B296F889B096F88AE0B6F8D6
:102610008E5081460022B246EC4840F2E63630F950
:1026200012C0ACEB050000F2F313B34204D800284B
:1026300004DCA5EB0C0001E04FF4FA7080B2022A32
:1026400033D0BBF1000F06D0834503D2A0EB0B00C3
:1026500080B200E000206423B0FBF3F3DD4E06EB14
:10266000430736F91380B7F90270A7EB08066FF03D
:1026700018077B4300EB83035E43642396FBF3F36D
:10268000D24E4344223E26F812309AF8303043436B
:102690004FF4FA70B3FBF0F0C0F16400C0B200FB7D
:1026A00009F06423B0FBF3F015E0BEF1000F06D093
:1026B000864503D2A0EB0E0080B200E00020C34E9E
:1026C000223EB0809AF8313043434FF4FA70B3FBA6
:1026D000F0F0C0F164000AEB0208C0B298F80E6096
:1026E00064234643B6FBF3F6B84F7E3FBE5498F8DA
:1026F00022604643B6FBF3F0FB1CAC45985406DA67
:1027000003F1590030F812305B4220F81230521CAD
:10271000D2B2032A80D3BAF89000814201DA01468E
:1027200004E04FF4FA63994200DD194689B2091AB0
:102730004FF47A725143C0F5FA60B1FBF0F081B208
:102740006422B1FBF2F0A34B6FF018060C3303EBDD
:10275000400533F910307043B5F9025001EB8000A9
:10276000ED1A454395FBF2F0DFF86082994EA8F12F
:1027700022081844103EA8F80600707AD146A8F145
:102780007E05E8B39448B0F90010B5F91A00081AAC
:1027900006F000FC914906F0F6F9914906F029FA95
:1027A000074607F023FA8346384607F0D5FF8246EE
:1027B0004746B8F9000006F0EDFB5146009006F0E0
:1027C000E2F98046B7F9020006F0E4FB59460190B1
:1027D00006F0D9F9414606F07EF906F0FAFB80468C
:1027E0005146019806F0CFF982465946009806F006
:1027F000CAF9514606F0C1F906F0EBFB388000E05B
:1028000001E0A7F802800220FEF73BFE002750B34C
:10281000E878401CC0B20621B0FBF1F2E87001FB81
:102820001200B8B902F0D5FF29796A4A01F007030E
:10283000703A491C22F813002971002032F8101058
:10284000401C2144C0B28CB20828F7D3E00800F045
:1028500090FE2872287A298C884203D899F8801033
:10286000814201D9AF7001E00420A870A87802F07D
:10287000A1FD5C48534C008818B10120FEF7ECFD27
:1028800010B95948008820B1206880F00800206005
:1028900014E0B178082011B14A49091D0860717827
:1028A00011B14849083108604FF40060FEF7E9FDB6
:1028B00020B1707800B1012002F06DFE8020FEF79B
:1028C000E0FD48B1E96BA86A411A05D44CF25031D9
:1028D0000844E86304F07AFAA96BA86A411A03D4A1
:1028E000717BF9B10120B07001F088FC1020FEF777
:1028F000B3FD68B1296CA86A411A09D4697A05291F
:1029000006D33A4908442864206880F0100020600B
:102910003748C16800290ED002B02C48BDE8F05FEE
:1029200084380847B770216881F008012160314977
:102930000844A863D8E7BDE8FC9F10B5244C2044A8
:1029400090F8810003F014FFA0F2EE2140F2DD5276
:10295000914201D3B4F88E0010BD2DE9F0471B4E13
:102960000024A03E1B4F7079DFF86080401C603F60
:102970007071A14607F14005316B20468847727996
:1029800007EBC40102F0030221F8120025F81490AD
:102990005FF0000035F8143031F81020401C1A4464
:1029A000C0B225F814200428F4D335F91400801C93
:1029B000C11700EB9170801025F81400414638F9DA
:1029C000142019E00C0C014014080140DC01002027
:1029D000040500209C08002044020020DB0F494031
:1029E000000034430002002002020020F0490200EF
:1029F0000409002020A10700D21E904202DA821CA6
:102A000021F8142031F91420D21C904202DD801EDE
:102A100028F81400641CE4B2082CADD3BDE8F0879C
:102A20002DE9F04F002085B08346019007460490C1
:102A300002F003FC08B1FFF790FFDFF808A44FF0A5
:102A40000005DAF82810DAF84800081AFE4C7BD4A2
:102A500044F6206211440820CAF84810FEF711FD20
:102A600008B9FFF77AFF4FF40070FEF70AFDDFF8B0
:102A7000D49309F1A00978B3DFF8D083BAF90C1028
:102A800098F8956006EB860C8C451DDA6078D8B115
:102A9000B8F98E3000204A4622F81030401CC0B2EF
:102AA0000328F9D3B8F89800A9F8060098F896001A
:102AB000304400EB800250468A4201DA657025708E
:102AC000C289521CAAF80E208C4502DA627802B93B
:102AD0002570491CAAF80C10DC48B9F9063001260B
:102AE000B0F890108B426EDAD648DFF860836A3017
:102AF0000580458085802638058045809AF8062027
:102B0000521CD2B28AF80620B9F90400884205DACC
:102B1000B9F90200884201DA607830B10420FEF78A
:102B2000B0FC70B3607880B139E0142A0BD1C8488A
:102B30004FF47A7101804FF48070FEF7A2FC0028F8
:102B400001D001F067FECDE0F3E1B9F90410B8F867
:102B500090204846914222DAB0F90210B8F892204B
:102B600091421CDDB9F90000904218DD9AF8061078
:102B70005046142904D1418A21B14582AAF8146033
:102B8000B0E00CE0C18B21B10021C18319B1022159
:102B900002E00121F9E703218AF80010A2E0B8F869
:102BA0006C10404681B1A8483230807938B1207825
:102BB00028B1A84866700188AAF81A1090E06078D9
:102BC000D0B365708CE038E0B9F90410B0F890200B
:102BD000CC46914207DB90F89430012B0BD1BCF925
:102BE0000030934207DA62782AB19AF80600142876
:102BF00078D1657076E0B0F89220914207DCBCF99C
:102C0000001091426CDD98F89400012868D1B9F960
:102C10000200904264DA607870B98D48008858B933
:102C2000A07848B19AF8061014295BD189496670DA
:102C30000988AAF81A1055E052E0DFF810824846D9
:102C4000B8F8922093424DDD63787BBBB0F9043035
:102C50008B420CDAB0F902C08C4508DA9AF806000B
:102C600014280FD17C4B4FF4C8721A800AE09342AB
:102C70000CDDB0F902308B4208DA9AF8060014280D
:102C800000D1A673401C8AF806002BE0B0F9023090
:102C9000934203DDB8F84400801C04E08B4206DA5E
:102CA000B8F84400801EA8F844000FE01AE0B9F913
:102CB0000000904203DDB8F84200801C04E0884226
:102CC0000EDAB8F84200801EA8F842000120FEF794
:102CD0003CFA8020FEF7D5FB20B104F0D8F801E0E3
:102CE0008AF806500420FEF7CCFB28B3BAF81E2061
:102CF0005046322172B1627862B1544AB9F9063055
:102D0000B2F89020934205DD4F4A323292790AB9E7
:102D10000182C5834C4A3232527A32B1C28A438A26
:102D20001A4309D1AAF8101006E0418A21B161784E
:102D300011B94582AAF814600020CE4640F2A4687A
:102D40000EEB4001B1F908C040F214518C4501DA94
:102D5000012100E0002100EB400901FA09F1ACF289
:102D60001552B2F5C77F01D8012300E0002309F115
:102D7000010293401943C44501DD012300E0002313
:102D800009F10202934019433943401CC0B28FB28B
:102D90000428D5D3DFF8B080DFF8B090002008F128
:102DA000320800BF09EB4001B1F86010394000D093
:102DB000012108F80010401CC0B20F28F2D398F887
:102DC000000038B999F8950000EB8001BAF90C00C1
:102DD00081420BDA0120FEF73FFB38B1E07830B9D1
:102DE0001848443005804580E67000E0E57098F8AA
:102DF000010038B1207930B912484430058045804F
:102E0000267100E0257198F8060000B92670E17877
:102E1000102009B9217909B1104901E00F49091FB2
:102E200008600220FEF718FB28B398F8020018B3D8
:102E3000A07900BB0A480B49A671006808600148E8
:102E40007E3011E03C0100208C08002004050020A9
:102E5000020200204402002000020020140C014065
:102E6000EC000020F0000020C188FF48AAF81810EC
:102E70000580FE48058000E0A5710420FEF7ECFA0D
:102E8000D0B198F80310404639B1617931B9F849A9
:102E900066710A88F7490A8000E06571817A19B184
:102EA000617A11B9667200E0657298F80E0018B187
:102EB000EF480188AAF81A101020FEF7CDFA40B3A7
:102EC000E07A30B39AF809005746052823D398F8DA
:102ED000070048B1E07940B9E749E671081F02F000
:102EE000E2F80220787000E0E57198F8080088B1F7
:102EF000207A70B9E04A26720C3A02F1100110688B
:102F00000860506841F8040F02F1100002F0CBF89D
:102F10007E7000E0257298F8090008B1A67200E002
:102F2000A57299F80500082801D00E2816D16572FF
:102F300014E09AF90700C21700EB927222F0030224
:102F4000821A00F101008AF8070047D0012A4DD00B
:102F5000022A53D0032A5AD08AF8075003F099FC6A
:102F6000C649CAF8280056468A8912B1F36CC31ABA
:102F70007ED41044F064FEF7EAFC03F08AFCB062F1
:102F8000F16A411A7181F0620420FEF765FA20B3FC
:102F9000B9491639B1F9042002F145008A2843D80D
:102FA000607998B3B2480388B2480088181A00B212
:102FB00010F1B40F02DC00F5B47000B2B42802DBEB
:102FC000A0F5B47000B2637B3BB1AC4B9B7D434337
:102FD0001E2093FBF0F0101A888029E00420FEF7F1
:102FE0003BFA0028BAD000F04AFDB7E70220FEF70E
:102FF00033FA0028B2D000F0C8FBAFE70220FEF79A
:103000002BFA0028AAD0FEF788FDA7E70CE00820DD
:10301000FEF722FA0028A1D000F0D0FD984896498A
:103020001E390088888099E791480188914801807D
:103030000220FEF711FAA8B1A07998B18E4BB6F92B
:103040001820163BB3F90610881A002800DC501A25
:103050008A4991F88B10884200DDA5718348008869
:103060001044D8801020FEF7F7F9E8B3E07900E0CB
:10307000D0E108B9207AC0B3207BB0B37C4EB6F95A
:10308000000005F087FF7F4F394605F07CFD07F013
:1030900063FB0090B6F9000005F07CFF394605F0AF
:1030A00072FD06F0A3FDDFF8D4818246724F98F8D6
:1030B000EF00DFF8D491443FE8B33E1DB7F90200BA
:1030C000B6F90210401A01F048F998F8EF10494299
:1030D00088420DDBB7F90200B6F90210401A01F080
:1030E0003CF998F8EF1001E065E003E0884204DD68
:1030F000084609E001F0AEFF5DE0B7F90200B6F95D
:103100000210401A01F029F9718808447080B7F95B
:103110000000B6F90010401A01F01FF998F8EF10FE
:10312000494288420CDBB7F90000B6F90010401A9A
:1031300001F013F900E046E098F8EF10884201DD55
:10314000084606E0B7F90000B6F90010401A01F091
:1031500004F93188084400B2308005F01BFF804636
:10316000009905F010FD0746B6F9020005F012FFC0
:103170005146039005F007FD4FEA070105F0FDFCFD
:103180004F46494605F035FD05F023FF3A4E5146BE
:10319000603E3080404605F0F6FC8046009903987A
:1031A00005F0F1FC414605F096FC394605F021FD9D
:1031B00005F00FFF708030491639B1F90200002880
:1031C00014DD034613E0B7F9000005F0E3FE804686
:1031D000009905F0D8FC0646B7F9020005F0DAFEC2
:1031E0005146039005F0CFFC3146C7E743422249E0
:1031F0001639B1F90010002901DD0A4600E04A4203
:10320000934203DD002806DC404204E0002901DD92
:10321000084600E04842DFF860800FFA80FE94F82C
:1032200004A0E278A8F13C08002008F10C0412B9CF
:10323000BAF1000F5ED0022859D20F49603931F936
:1032400010304A3131F9101003EB41010F4B994214
:1032500002DB5B42994200DD19460D4BDFF81CC0D2
:1032600033F81030C91A15E0BE000020BC00002061
:103270004402002046020020D00100200405002066
:103280002801002035FA8E3C000020410CFEFFFF93
:10329000CC0000200CEB40036426B3F842309CF8CD
:1032A000297019449CF8153009B24B4393FBF6F38F
:1032B0007E421BB206EB86069E4203DC07EB8706C6
:1032C0009E4200DA33460293544B33F91060314486
:1032D000534EB14203DB7642B14200DC0E4631B2BE
:1032E00023F810109CF81F305943091301910AB1BB
:1032F000022833D149494B4E3A3106EB000C31F9E3
:1033000010309CF80E6003EB8301090191FBF6F18C
:10331000454E9B4636F91070404EC91B263609B201
:1033200036F910301944414B994202DB5B42994215
:1033300000DD194607F5207726F81010B7F5A06FC5
:1033400001D926F8105036F910107D2391FBF3F1C6
:103350009CF818305943891109B20491BAF1000F51
:1033600017D0022815D20299CEF5FA7707FB01F3A0
:103370000BFB0E314FF4FA7C019E91FBFCF107FB35
:1033800006F3049E09B206FB0E3393FBFCF31BB25B
:1033900007E022B1022802D2DDE9013101E0049BFD
:1033A00059469946204B5027DFF870C033F910601A
:1033B0001A4B0CF11A0C223B1B5C734393FBF7F383
:1033C000CB1A38F8101028F81060711A3CF8106009
:1033D00034F8107024F8106037440F442CF81010A3
:1033E000ACF139013FB2095C4B447943A3EB611363
:1033F0000CF1120121F81030401CC0B20328FFF478
:1034000016AFFEF7B8FEFEF769FE05B0BDE8F04F57
:10341000FEF792BE05B0BDE8F08F000080010020ED
:10342000F0D8FFFF04050020F800002080C1FFFF56
:103430002DE9F843F94CFA4900252F4694F8542019
:10344000A1F1100003F0DBFD08B101250CE0F44808
:1034500003F089FF08B1012706E0F14802F051FFAF
:1034600010B9032003F0BDFAEE4E4FF0000800BF84
:1034700094F8460030B1012804D0022814D0032863
:1034800028D11FE08DF800804FF44870E449ADF872
:1034900002001039684602F02FFA08B1012030709E
:1034A00094F84600012815D065B1DD4994F8542000
:1034B000A1F1100003F0A3FD0220307094F8460043
:1034C000022812D0D648103803F04EFE10B1032067
:1034D00030700AE0307840B994F8460010B184F8B2
:1034E0004680C5E70120FDF7C4FFCD48103004F049
:1034F00017F838B9CA48103002F092FA10B9022011
:10350000FDF7B7FF0120FDF7A7FF18B1C448103839
:1035100000688047C2480068804727B1B4F84A0075
:1035200003F03AFF04E01DB9B4F84A0002F0FFFED0
:1035300002F088FB10B90420FDF79BFFB4F94000AE
:10354000642290FBF2F102FB11000CB205F022FDA7
:10355000B54905F018FB0546204605F01BFD294638
:1035600005F0B9FAB14905F00EFBB1490860BDE8B4
:10357000F88370B50546A94890F87E0005F013FD64
:103580000446284605F00FFDAA4905F0FCFAAA49B1
:1035900005F02FFB214605F0F6FA05F033FD80B269
:1035A00070BD70B500252C4602F013F905440A20C1
:1035B00003F092F9641C202CF6D3C5F34F10FFF7EB
:1035C000D8FF964A022192F87F3000BF03FB01F436
:1035D000844202D8491C0629F8D39848017092F811
:1035E000800048439649088070BD2DE9F047DFF818
:1035F0003492944E894CB9F804200025AAB3884926
:1036000000204FF4C87C3439C846624501D141F8E6
:10361000205051F8203036F910703B4441F82030EA
:1036200026F8105004EB4003401C9D860328ECDB79
:10363000012A15D1086890FBFCF0A086486890FB31
:10364000FCF0E0868868B8F8081090FBFCF0401A9F
:103650002087A4F84250A4F844500120FDF775FDDE
:10366000B8F80400401EA8F804000420FDF709FF84
:10367000002870D0744BDFF8ACC169491A880CF18E
:103680001C0C2839ACF11208322A05D0EAB300200C
:103690009A46322A12D013E0A08EACF80000E08ED9
:1036A000ACF80200208FACF80400B4F84200A8F88F
:1036B0000000B4F84400A8F80200E8E741F8205000
:1036C00051F8203036F910703B4441F8203026F88C
:1036D000105004EB4003401C9D860328D9DB012ACF
:1036E0001AD15A485A4B058001201880594B0220A4
:1036F0001870BCF80000A086BCF80200E086BCF898
:1037000004002087B8F8000000E008E0A4F84200B8
:10371000B8F80200A4F84400521EAAF800204E484F
:103720000288012A17D105800A68322092FBF0F244
:10373000A2864A6892FBF0F2E286896891FBF0F17A
:10374000B9F80800081A2087A4F84250A4F8445099
:103750000120FDF7FAFC3088A18E401A3080708875
:10376000E18E401A7080B088218F401AB080BDE889
:10377000F08710B52A4C3348103C61688847A1682F
:1037800030488847BDE810402FE770B53348254CD6
:1037900000682169411A2CD42061214DA078103590
:1037A00040B301282DD0022831D0032821D16869E7
:1037B0008047A869804705F0EDFB294905F019FA13
:1037C00005F053FC4FF00052264B06F0CFFA0022D2
:1037D000254B05F0FDFA0022244B05F0FCFA05F01C
:1037E00025FC234908600020A070A88821690844AE
:1037F000206170BDA8688047A078401CA070288810
:10380000F4E7E8688047A078401CA07070BD286984
:103810008047A078401CA0706888E7E70405002076
:1038200004090020FC0100208988883C0000204118
:10383000C80000203333534000F07F45F3010020DF
:103840005C010020100100204C01002052010020EA
:103850004E0100203C0100205001002064010020A6
:1038600080E6C547965BC83F0000F03F1AE950412B
:10387000E80000202DE9F047D24FD34ED34CF88812
:1038800030B30025DFF84883A9464FF47A7AF988E7
:10389000514501D148F8259058F8253034F915C024
:1038A0000129634448F8253024F8159026F815902E
:1038B00008D193FBFAF026F8150001220F210A2007
:1038C000FEF75AFE6D1C032DE1DBF888401EF880E0
:1038D000BC4D002015F1220534F8101036F81020E8
:1038E000891A09B224F8101035F91020A2F548738E
:1038F000994201DA1A4604E002F54872914200DC6E
:103900000A4624F8102025F81020401C0328E3DB89
:103910002DE710B5AE4CAD481C3461688847A168EE
:10392000AA488847BDE81040A4E7A64810B528304B
:1039300002F0DEF9A348A749283082880A8002886D
:1039400052424A8040884042888010BD2DE9F04FA5
:1039500085B06020029040F2FE20039040F2C92022
:10396000049000279C483D46009002F07EF9954C5B
:1039700000203C34DFF864A220606060DFF860B2B1
:10398000A0604CE07F1C029802F08AF9642002F0EB
:10399000A3FFFFF7CAFF0A2002F09EFF8D4EB6F983
:1039A000000005F0F7FA8046039805F0FCFA41465E
:1039B00005F01FF920F00049B6F9020005F0EAFA17
:1039C0000646049805F0EFFA3146019005F011F92A
:1039D00020F000464146019805F00BF97F4920F0A0
:1039E0000048C94309EB01007E49884217D2564579
:1039F00015DD5E4513DAD04511DDD8450FDA6D1CB3
:103A00004946206805F067F820603146606805F097
:103A100062F860604146A06805F05DF8A060142F70
:103A200002D2052DAED301E0052D1BD3284605F0AB
:103A3000BAFA05462068009905F0A5F8294605F070
:103A4000D8F820606068009905F09DF8294605F0D7
:103A5000D0F86060A068009905F095F8294605F057
:103A6000C8F803E04FF07E5020606060A06002F074
:103A70002DF954490120487005B0BDE8F08F2DE9BB
:103A8000F04759484F4D00686969411A75D4574944
:103A900008446861FFF749FF4E4CB4F9000005F097
:103AA00079FA05F13C06316805F06DF805F091FAF8
:103AB00000B220808146B4F9020005F06BFA71680B
:103AC00005F061F805F085FA00B260808246B4F92D
:103AD000040005F05FFAB16805F055F805F079FAD1
:103AE000DFF80C810FFA80FCA4F804C098F80E00EF
:103AF0000027404A05F12E018B1D88B16869A86135
:103B00005FF0000002EB4006778734F8106021F880
:103B1000106023F81060401C0328F3D388F80E705F
:103B2000687858B1568FA9EB06002080968FAAEBD3
:103B300006006080D08FACEB0000A080A869002850
:103B40001BD06E69301A2C4EB04217D22B48026837
:103B500082F008020260002034F9102031F9105080
:103B6000AA4201DA21F8102033F91050AA4201DDEF
:103B700023F81020401C0328EED3F8E50020AF61A5
:103B800031F9104033F910502C4404EBD47402EB9B
:103B900040056410401C6C870328F1D3BDE8F04752
:103BA0000120FDF7D2BA10B5012003F024FB082054
:103BB000FDF75AFC12490020088010BD104803F0A0
:103BC0006DBB0000FC010020220100200A01002042
:103BD000E80800201C01002059021B3F3333333F0B
:103BE0006666A63F3233730064010020A0860100A0
:103BF0008C0800200405002080C3C9010C0C014082
:103C00002801002070B5FA4C0546C0B2A07003F040
:103C10000AF8E079A1784840E071C5F30720A07068
:103C200003F001F8E079A1784840E071C5F307405E
:103C3000A07002F0F8FFE079A1784840E071280E0A
:103C4000A07002F0F0FFE079A1784840E07170BD0B
:103C500070B5E74C0546C0B2E07002F0E4FFE079D1
:103C6000E1784840E071C5F30720E07002F0DBFF27
:103C7000E079E1784840E07170BD10B5044602F08B
:103C8000D2FFDB48C1796140C17110BDD84AD94823
:103C9000117A405C491C1172704700B5FFF7F6FFBE
:103CA0000346FFF7F3FF03EB002080B200BD10B521
:103CB000FFF7F3FF0446FFF7F0FF04EB004010BDF1
:103CC00070B504460D462420FFF7D7FF4D20FFF7BF
:103CD000D4FF0CB1212000E03E20FFF7CEFFC44C02
:103CE0000020E0712846FFF7C8FF607ABDE8704009
:103CF000C3E701460020E3E701460120E0E7BC48B6
:103D0000C079BAE710B5044603E000BFFFF7B5FF7E
:103D1000641C20780028F9D110BD02F0D7BE2DE92F
:103D2000F05FB348B44DDFF8D492407AB44EDFF878
:103D3000D4A2DFF8D4B2B54FDFF8D482B54C7328E3
:103D400078D00DDCA0F164000F282BD2DFE800F062
:103D500091A1FEFDFCFBFAF9F8F7F6F5F4F3F20099
:103D6000CC2869D010DCC82822D006DC74287AD090
:103D7000752879D0762815D104E2C92825D0CA281B
:103D80003DD0CB280ED14AE0D0286ED006DCCD281D
:103D90006CD0CE286BD0CF2804D112E0FA2867D09F
:103DA000FE2875D00020FFF7A7FFBDE8F05FA6E76B
:103DB00000244546FFF771FF25F81400641C082C09
:103DC000F8D30020FFF795FFEFE7FFF75FFFE872FA
:103DD000FFF75CFF89F80000FFF769FF3060FFF72D
:103DE00066FF7060FFF759FFAAF80000FFF755FF64
:103DF000ABF80000387840F002003870E1E70023AB
:103E0000FFF744FFE518A873FFF740FF2876FFF798
:103E10003DFF5B1C85F822000A2BF1D3D1E700257A
:103E2000FFF73BFF04EB45016D1CA1F860000F2D6F
:103E3000F6D3C6E79AE1FFE7FFF728FF04F82C0F57
:103E4000FFF724FF6070FFF721FF2071FFF71EFFCF
:103E50006071FFF71BFFA071FFF718FFA070FFF75D
:103E600015FFE070ADE76FE173E1AAE1ADE1B1E10B
:103E7000B3E10720FFF73DFFD320FFF7FEFE607997
:103E8000FFF7FBFE0020FFF7F8FE4FF0004061E077
:103E9000A7E10A20FFF72DFF5F48008800B2FFF777
:103EA000D7FE02F063F900B2FFF7D2FE0120FDF762
:103EB000D3FA04460220FDF7CFFA44EA4004042076
:103EC000FDF7CAFA44EA80041020FDF7C5FA44EA77
:103ED000C0040820FDF7C0FA44EA0010FFF7B8FE5E
:103EE000E87829796A7940EA4100A979890041EAAC
:103EF000C2010843697840EA81114848027941EAE1
:103F00000211427941EA4211EA7941EAC2112A7A60
:103F100041EA02216A7A41EA8221AA7A41EA4221EF
:103F2000C27A41EAC221027B41EA0231427B41EA84
:103F300042310CE015E1F8E0E4E0CBE0C2E0BBE0A8
:103F4000A2E090E076E045E036E027E005E0807B07
:103F500041EA8030FFF756FE27E71220FFF7C9FE3F
:103F60002F4D002435F91400FFF772FE641C032C5A
:103F7000F8D32C4D002400BF35F91400FFF768FE7C
:103F8000641C032CF8D3284D002400BF35F914001D
:103F9000FFF75EFE641C032CF8D306E71020FFF742
:103FA000A8FE224D002400BF35F91400FFF750FE93
:103FB000641C082CF8D3F8E61020FFF79AFE1C4D7D
:103FC000002400BF35F91400FFF742FE641C082CE2
:103FD000F8D3EAE61020FFF78CFE00244FEA08052C
:103FE00035F91400FFF734FE641C082CF8D3DCE626
:103FF00048020020300900208C08002045010020E4
:10400000C4010020F8010020FA010020EE01002088
:10401000DC0100200405002046010020BE0800202D
:1040200016010020F80000201C0100202C010020B7
:10403000540700200E20FFF75CFEE87AFFF71DFE14
:1040400099F80000FFF719FE3068FFF7DBFD706894
:10405000FFF7D8FDBAF8000000B2FFF7F9FDBBF892
:10406000000000B225E00520FFF743FE9E480088CF
:1040700000B2FFF7EDFD9D48B0F90000FFF7E8FD45
:10408000387800F0010094E00820FFF732FE984DE8
:10409000002400BF35F91400FFF7DAFD641C022C80
:1040A000F8D39448B0F90000FFF7D2FD9248B0F978
:1040B0000000FFF7CDFD78E60420FFF71AFE8F48D9
:1040C000006847E70320FFF714FE8D480078FFF7EC
:1040D000D4FD49E00720FFF70CFE14F82C0FFFF782
:1040E000CCFD6078FFF7C9FD2079FFF7C6FD607948
:1040F000FFF7C3FDA079FFF7C0FDA078FFF7BDFD76
:10410000E07856E01E20FFF7F4FD00256619B07B2D
:10411000FFF7B3FD307EFFF7B0FD96F82200FFF702
:10412000ACFD6D1C0A2DF1D33FE61E20FFF7E1FD2B
:104130005FF0000504EB4500B0F96000FFF788FD73
:104140006D1C0F2DF6D330E66D20FFF7D2FD6D48C4
:1041500004E02F20FFF7CDFD6A486E30FFF7D2FD57
:1041600023E60220FFF7C5FD0020A2E70820FFF7A5
:10417000C0FD0024601CC0B2FFF77FFD641C082C4A
:10418000F8D312E6FFF782FD04460C20FFF7B1FDDD
:1041900094B1102C8FD11020FFF76FFD5A4C20687E
:1041A000FFF730FD6068FFF72DFD0020FFF750FDA1
:1041B0000020FFF762FDF8E50020FFF75EFD534C9D
:1041C000EDE70120FDF70CF9FBE551494FF4C8700C
:1041D0000880F6E50120A873F3E50020FCF7B5FFA1
:1041E000EFE50820FFF785FD4A4D002435F914005E
:1041F000FFF72EFD641C042CF8D3D6E570B5464CB1
:104200000025607810B3BDE87040FCF773BD00BFB7
:1042100002F0FCFCA17951B101291CD002291FD068
:10422000032923D004292CD0052942D12FE02428AA
:1042300003D00021A17149B901E00121FAE7232847
:1042400002D0522835D102E0FCF754FD31E00120C4
:1042500002F0EAFB2DE04D2804D10220A07128E0F5
:104260003C2801D00020F9E70320F7E740281FD8B9
:10427000607125712572E0710420A0710120207009
:1042800017E06072E1794140E1710520E6E72179AC
:104290006279914207D2E2794240E2711F4A50545A
:1042A000491C217105E0E179814201D1FFF737FD19
:1042B000A57102F095FC0028AAD16078002811D1E0
:1042C00002F08EFC00280DD14FF40060FDF7D9F804
:1042D000002807D012484078002803D0BDE870407D
:1042E00001F06AB970BD0000F4010020F601002061
:1042F000CC0000204402002056010020EC000020E9
:104300004401002018B50008D4010020CC01002091
:1043100000020020B20100204802002030090020E5
:104320008C08002070B50446FE4D09E002F0FBFC4D
:1043300095F8E400012802D1042002F0CDFA641CB3
:1043400020780028F2D100BF02F0FFFC0028FBD04B
:10435000BDE870401E2002F0BFBA44F250618842AE
:1043600001DDA0EB4100F049884202DA48F6A041A5
:10437000084470472DE9F047054650680E4614463C
:104380009946281A04F006FE316804F032FC2061D8
:10439000A768394604F0F1FB8046E24890F8EE0049
:1043A00004F001FEE14904F0EEFB01464FF07E50BF
:1043B00004F01FFC3668314604F08DFB01463046A0
:1043C00004F017FC414604F0DEFB394604F083FBA1
:1043D0002061C4E901500146D9F8080004F0D3FB7C
:1043E000BDE8F04704F0F5BD70B50E4614461D4615
:1043F00004F0D0FD696804F0C6FB316804F0C3FB2B
:10440000216804F068FB01462060E86880F0004005
:1044100004F068FE03D2E86880F0004007E0E96835
:10442000206804F05FFE01D2E86800E020682060A8
:10443000BDE8704004F0CDBD70B5BD4CD4E90D01B0
:10444000401AFFF78AFF0028D4E90D01A0EB010014
:1044500002DDFFF782FF02E0FFF77FFF404241F2FB
:10446000941188422ADAD4E90D01401A04F092FD31
:10447000B04904F088FB0646E06B04F094FD054665
:10448000304606F069F9294604F07DFB04F0A1FDF1
:1044900000B2A9492082884202DB4942884200DDFD
:1044A0000846616B084448F6A0416064884200DD1C
:1044B000401A002800DA0844606470BD606BFBE7B6
:1044C0002DE9F04F87B00646FFF7B6FF984842F255
:1044D0002831406C081A04F05DFD964904F053FB46
:1044E000044605F083FB0590204606F035F9904D13
:1044F000049000243035DFF840B2DFF84092DFF856
:1045000040A2304604F046FD009089481A3030F948
:10451000140004F03FFD064604A850F8241000984B
:1045200004F031FB314604F028FB04F052FD00B2E8
:10453000844925F81400884202DB4942884200DDA4
:1045400008467E4925F81400603900F0D3FD04EBDD
:1045500084067A4B7649074609EB860835F914003C
:10456000603B42462831FFF73FFF744B70490744D8
:1045700035F91400603B42462831FFF7FBFE384412
:1045800000B22AF81400584501DA584604E040F613
:10459000B832904200DD10462AF81400674859F8F6
:1045A00026102838641C40F82610022CADDB07B01A
:1045B000BDE8F08F2DE9F05F5D4E0024DFF87C91BF
:1045C0005036DFF87CB1A6F1360AA9F1280900BF00
:1045D0005A4956F82400803900F08CFD3AF814103E
:1045E000534F401A3037554900B227F8140070393C
:1045F00000F080FD054637F9140056F8241004EB4E
:104600008407084409EB870188460A464B4B484912
:10461000703B2831FFF7E8FE2844484B44492BF80B
:1046200014005D4656F82400703B42462831FFF7DF
:10463000A1FE4549884202DB4942884200DD084626
:104640003AF914103131622900D8002035F81410DD
:10465000084400B2384925F81400884202DB494278
:10466000884200DD084625F81400344859F8271020
:10467000641C40F82710022CAADBBDE8F09F70B53F
:104680000446086819681546401A04F083FC284956
:10469000C96A04F078FA04F09CFC014624485030C2
:1046A000416021682A68891A016070BD2DE9F041D6
:1046B0000E46DDE90685116800681F46081A04F0F9
:1046C00069FC044638683168401A04F063FC1849F4
:1046D000C96A04F058FA0646014604F054FA07463F
:1046E0002146084604F04FFA394604F0F4F906F082
:1046F0001FF9164904F047FA04F084FCC8F80000DA
:1047000084F00040314605F047F9114904F03BFAC6
:10471000104904F0E0F904F05CFC286000281FDA7E
:104720001AE0000004050020B0B9FFFFDB0FC9400C
:1047300054020020D302373948F4FFFF100A00204A
:104740008C01002018FCFFFF30F8FFFF2C7D8E3F0E
:10475000A00CB34500A00C4648F6A04108442860D0
:10476000BDE8F0812DE9F047FB48FA4CD0E900653F
:10477000617804F14808A1B34FF07E50A16A04F0BB
:1047800038FA8246D8F80400281A04F003FCE16ADB
:1047900004F0F9F9514604F0F6F904F01AFC07B2F6
:1047A000D8F8000004F11A09301A04F0F3FB51465E
:1047B00004F0E9F904F00DFC02B204F12400B0F9B0
:1047C0000210394401EBD1714910A9F80210B0F977
:1047D00000301A4402EBD2725210A9F80020418036
:1047E000028001206070C8E90065BDE8F08710B55F
:1047F000044604F0CFFB002C01DC80F00040D749D8
:1048000004F0F7F9D64904F0BEF905F0EFF9D14903
:10481000C86210BD10B5D34CE07A002811D0D24840
:10482000007805280DD3CC49D04A08681060496843
:104830005160FFF7DCFFCE48C6490088888201201E
:10484000207310BD70B5C349C64B01248D7AC94889
:104850000022022D07D0032D15D0062D21D0122DB8
:1048600031D0002070BDBC4D46686E6086682E60F9
:1048700000694FF47A7590FBF5F0BF4D2880C87A37
:10488000D8724C732AE04479E40702D000790328F7
:1048900003D00020C87210B120E00120FAE7DA72DC
:1048A0001CE0C47AE40702D0847A032C03D00024ED
:1048B000CC7214B102E00124FAE7DA72AA4B90F844
:1048C0002F0018700AE0AD4D43692B80806942F2D9
:1048D000107390FBF3F0AA4B18808C73487B8B7B92
:1048E0001840BFD04A738A73012070BD2DE9F0478C
:1048F00098494FF000090A464E7AD579137A2C1858
:10490000B2F816C04FF00108E4B24A46092E56D25A
:10491000DFE806F0080510161D2434444A0062281A
:1049200003D04A72B52802D049E0022034E081F871
:10493000098044E003224A720873C87108723EE09D
:1049400004224A72CC71E2180A72887237E005229A
:104950004A72CC71E2180A72C88230E006254D72A4
:104960000CEB0020CC71234480B20B72C882B0F5EE
:10497000007F01D9CA824A720A8320E0CC71E21812
:104980000A720A8B402A01D27A4B9854521C90B278
:104990000883604513D10720487210E008234B724A
:1049A00085420CD04A720AE04A72834207D17548A8
:1049B00080F80080FFF746FF08B14FF00109484634
:1049C00013E770B5034600200246054611E02E2C81
:1049D00004D1521C00290FD054181D559C5C00EBCB
:1049E00080004000A4F13006092E01D83038204460
:1049F000521C9C5C002CEAD170BD2DE9F0410025D1
:104A000080462E462F46044603F0ACFF016800E0C6
:104A1000641C2078085C2028FAD0404609E01DB1CB
:104A200005EB85025206150E10F8012B303D2A4485
:104A3000D5B2221A022AF2DC09E01EB106EB860288
:104A40005206160E10F8012B303E3244D6B2844284
:104A5000F3D820782E280ED1641C002007EB8702A3
:104A6000570022788B5C202B02D1303F1744641C06
:104A7000401C0428F2DB44480621464307EBC700EC
:104A800000EB071006EB8000B0FBF1F03F494D430F
:104A900000EBC51064E62DE9F04700272D4C0546D4
:104AA0003E464FF00109242815D032482146F038FF
:104AB000C9782C2D13D02A2D11D022460D2D5279D4
:104AC00047D00A2D45D00F2902D24554491CE17028
:104AD000002A73D0ACE0A670E6702671A8E04654B8
:104AE000A178B046324629B1A279012A21D0022A02
:104AF0007CD093E0A2710178472907D141785029F1
:104B000004D18178472902D0522909D086E0C178A2
:104B1000472904D10079412801D184F806907DE02D
:104B2000C1784D297AD10079432877D10220A0712C
:104B300074E0094E02292BD003292DD0042932D04C
:104B4000052934D006293AD0072941D0092947D070
:104B500064E07AE054020020C40100208096184BE3
:104B600035FA8E3C8C08002045010020CC01002045
:104B700044020020600A0020F8010020FA01002011
:104B8000F0010020F201002040420F002D31010011
:104B9000F848FFF732FF04E0007853283ED1306830
:104BA000404230603AE0F348FFF727FF04E0007826
:104BB000572833D17068404270602FE035E00078AC
:104BC000302801D9012000E00020EB49C87225E01F
:104BD0000021E848FFF7F5FEE84908701EE005E00F
:104BE0000021E448FFF7EDFEE54916E0072902D071
:104BF00008290DD012E00121DE48FFF7E2FE41F264
:104C0000184148434FF47A71B0FBF1F0DD4904E0FC
:104C10000121D848FFF7D5FEDB490880A078401C69
:104C2000A07084F803802A2D0CD020796840207170
:104C3000A07910B1D54A82F800900FB1012800D0B8
:104C40000020D2E584F80590F2E772B18046007842
:104C500000F07EFA050198F8010000F079FA284486
:104C60002179C0B2884200D101276671E0E72DE9C1
:104C7000FF5FC749C0B291F8E41019B1012904D00F
:104C800002297DD1FFF707FF01E0FFF72FFE002883
:104C900076D0C0484FF0000B0178012910D00121D7
:104CA0000170B548C17A00296AD0B449097805294C
:104CB00066D38246407830B19AF80C1031B108E0E2
:104CC00080F800B0EDE78AF80CB002E008B1FFF719
:104CD000A1FDB1490523DFF8C88208789E46401C33
:104CE000B0FBF3F203FB12020A70AC49002091F909
:104CF000009000BFA84958F820306831A64C41F810
:104D00002030A849783493FBF1F144F82010A64CE8
:104D100000EB80054C4303EBC41342F2107493FB89
:104D2000F4F41FFA84FC9C4C403424F810C0914CDD
:104D3000C83404EB8505984C55F82260603454F86B
:104D4000207045F82230BE1B334444F8203093FBDA
:104D5000FEF3954C6442614303EBC1138E497031FD
:104D6000B9F1010F41F8203006D1ACF1020CBCF5CD
:104D7000797F01D848F82030401C0228BADB00E0D7
:104D80007BE001F09BFD844D296A401A04F00BF989
:104D9000864903F02EFFA86201F090FD2862A86A00
:104DA0004FF07E51884200DB0846A86203A902A8A2
:104DB0007F4BCDE9000146461A1F311D7848FFF7A9
:104DC00075FC02994FF06408B1FBF8F1794A54463A
:104DD0001180039991FBF8F0774908809AF80C004C
:104DE00018B9A2F800B0A1F800B0FFF7BBFC207A18
:104DF00010B9E079002840D067493446343101F1D8
:104E0000080000F11C07CDE900013B1D3A46311DA9
:104E10006348FFF74BFC231D614A391D3846FFF7F5
:104E20002EFC5E4C94F90000012828D0022824D1E1
:104E3000574E0121B6F9F40000F067F9FFF740FB87
:104E400096F8F0005D4A18B1696C91FBF8F010809B
:104E5000B6F8EC00E96B88420BD2D5E90D01401A97
:104E6000FFF77BFA002800DC404242F210718842D2
:104E700003DD01202070A88A1080BDE8FF9FFFF7A6
:104E800099FBFAE72DE9F047414C1234207804F001
:104E90008AF8DFF82C91494603F0ABFE354D2035FA
:104EA0002860A07A04F07FF8494603F0A2FE454E40
:104EB000EE606860607804F076F8434F394603F09E
:104EC00098FE10352860E07A04F06DF8494603F04A
:104ED00090FE6860607D04F066F8DFF8D08041469F
:104EE00003F087FEC5E90206A07804F05CF83946B5
:104EF00003F07FFE10352860207B04F054F849460B
:104F000003F077FE6860A07D04F04DF8414603F0A1
:104F100070FEC5E9020668E42DE9F0470746002463
:104F2000FFF7B0FF00222949384601F0B6FE184EBF
:104F300096F8E400012802D0022849D0C0B1DFF879
:104F40005880002508F180084FF4964A08F11409AA
:104F500058F8250001F0E6FE57453BD0B7F5164F4F
:104F60003BD0B7F5614F4DD0B7F5E13F3AD14DE0B9
:104F70003EE00000700900208C0800204501002060
:104F8000F8010020FA010020F0010020F2010020C9
:104F900004050020EE010020540200203D01002005
:104FA000C401002080969800D3CEFEFF00007A4412
:104FB000D0010020F4010020F6010020460200206C
:104FC0000000C8420000FA44000020416F4C000875
:104FD0000424B4E759F8240002E009EB8400406897
:104FE000FFF7A0F90A2001F077FC6D1C052DAFDB5F
:104FF000384601F097FE96F8E40001280AD002280E
:1050000014D019E009EB84008068E9E709EB84001B
:10501000C068E5E7554D0024285D01F084FE0420BA
:1050200001F05AFC641C8C2CF6D305E050A0FFF76D
:1050300079F95CA0FFF776F94FF47A7001F04CFC37
:105040005D480078002804D0BDE8F0471020FCF748
:105050000BBAB5E42DE9F05FDFF86CA10024574FDF
:10506000DFF85C81DFF85C9125460AF1280B00BF70
:1050700027F8145028F8145004EB840629F814502B
:105080000AEB860000F06DF80BEB860000F069F883
:105090004D48503000EB860000F063F8641C022C91
:1050A000E6DBBDE8F09F7CB5484C026822600968E9
:1050B00061600068FFF79BFBA4F1240101F1080087
:1050C000434ECDE90001231D2246311D3046FFF736
:1050D000EDFAA4F15805331D686B68643246211D52
:1050E0002046FFF7CCFA686BA8633A48B0F8F200A4
:1050F00068827CBD10B50C4603F04CFF216803F0BC
:1051000042FDBDE8104003F064BF70B52F4C583C21
:10511000E26B21B1B0EB520F0BD3500809E0904283
:1051200000D310462B4900B2B1F8F210814200DBE7
:105130000846B4F9125000B2A84208DD2649A06A18
:1051400003F021FD03F045FF284400B2608270BDEA
:105150003038C0B2092801D9C01FC0B200F00F001A
:10516000704700210160416081607047B6B500085A
:1051700024504D544B3331342C302C312C302C31C5
:105180002C302C302C302C302C302C302C302C303F
:105190002C302C302C302C302C302C302C302A322F
:1051A000380D0A0024504D544B3232302C323030FE
:1051B0002A32430D0A000000F20100207001002095
:1051C000900100208C010020C0090020AC020020CA
:1051D000C4010020040500200000C84270B5374C0F
:1051E00001260546667001F054FBA168421AC4E925
:1051F000020241F288300021824200D9A170304A77
:10520000A07815540F2802D0401CA07070BD2D4806
:105210002670018070BD2C48032190F88C2027480F
:1052200012B1C170072101E00222C2700171012296
:1052300026494FF4E13001F030BD20480078704736
:10524000F0B51E4A1E4B11781C3BE9B11679D57892
:10525000DFF86CE0032100BF0EEB010717F8014CEB
:10526000EC4004F00F04072C08D21EF801C017F818
:10527000017C37400CEB072743F82470891CC9B226
:105280001029E9D3002111700F4907280FD2527855
:105290006AB10D4A91F88C10104490F8810053F8CF
:1052A000200039B14FF4777101EB500004E0B1F800
:1052B0008E00F0BD00F5777080B2F0BD08030020CD
:1052C000BC0A00204801002004050020DD51000830
:1052D0002DE9F0417E4C0746012520782E0380B948
:1052E00001F0ECFAA1683231884207D37948257081
:1052F000066001F0E3FAA060BDE8F08120780028A4
:10530000FAD001F0DBFAA16839448842F4D30020D6
:1053100020707048001F066001F0D0FAA0606E484F
:10532000017809B1491E01706570E5E7F8B5684D6F
:105330008DF800008DF801108DF802208DF80330F3
:10534000A8791DF8001044292FD04C292BD04D29C5
:1053500027D04E292CD032240026032806D274B13F
:105360002046FFF7B5FFA879032808D301F0A6FA75
:10537000A968001B884202D95748AE710670687848
:10538000012801D0002C0BD1A879032801D2401CA0
:10539000A87150496E70091F2E704FF4805008603C
:1053A000F8BD6424D8E7C824D6E74FF4FA64D3E7FD
:1053B0000024D1E72DE9F047DFF820A10546444C51
:1053C0009AF80B004FF00109002610B184F8029002
:1053D00000E0A6704FF40070FCF753F8404F18B38C
:1053E000404941484FF0020891F89530B0F900006B
:1053F00003EB830282420FDA97F801C0BCF1000F81
:105400000AD084F8049091F89610194401EB8101B8
:10541000814201DA84F80480824203DA797809B99A
:1054200084F8048000B926711020FCF715F840B10B
:105430009AF8071011B99AF8080008B1F87AA8B1DB
:10544000E6702079022814D0012817D0E0780128CE
:1054500017D0A078012817D0042D19D0022D1ED006
:10546000012D1ED0607901281ED022E084F803901F
:10547000E7E74E22442311464C200DE04D234C22F9
:1054800008E04D234E2201E04D235322532102E038
:1054900044234D224D215320BDE8F04746E74423E5
:1054A00005E044234E22F5E7787810B14E234D22D3
:1054B000ECE70948007818B1BDE8F047322007E76B
:1054C00004492670091F4FF480500860BDE8F0873A
:1054D00018030020140801403C010020BE080020F1
:1054E0008C080020040500204801002070B513201E
:1054F00000F0F3F8834C2068002800DC4042824D25
:1055000090FBF5F000B200F0F2F81B2000F0E5F897
:105510002068002800DC404290FBF5F042F2107653
:1055200090FBF6F106FB110000B200F0E0F823203A
:1055300000F0D3F82068002801DA532000E04E2064
:1055400000F0D5F8122000F0C8F86068002800DCF0
:10555000404290FBF5F000B200F0C9F81A2000F0CC
:10556000BCF86068002800DC404290FBF5F090FB3E
:10557000F6F106FB110000B200F0B9F8222000F0AD
:10558000ACF86068002801DA572000E04520BDE84B
:10559000704000F0ACB870B55C4D04462878844289
:1055A00009D014B14FF4165002E05948D0F8F80071
:1055B000FEF7B3FB2C7070BD2DE9F04701F07EF9CA
:1055C000524D6968401AC8287DD301F077F96860A8
:1055D0006878504F401CDFF84081DFF840916870D8
:1055E000002400BF04F12400C0B200F076F838882F
:1055F00003F0D9FC064638F9140003F0CBFC314621
:1056000003F0F7FA494603F0BEFA03F0E2FC00B2F9
:1056100000F06DF8641CE4B2032CE3D3102000F01A
:105620005CF83F4C6426206890FBF6F000B200F076
:105630005EF8212000F051F8206890FBF6F106FB9F
:10564000110000B200F053F8022000F046F835488F
:105650000A21B0F9000090FBF1F000B200F047F829
:105660005E2001F0E0FA68780521B0FBF1F201FB61
:10567000120040B91020FBF7EFFE20B1FFF736FF14
:105680005E2001F0D0FA6878192824D100206870D3
:1056900001F014F94FF47A71B0FBF1F43C25B4FB3E
:1056A000F5F6B6FBF5F005FB1067172000F015F8CE
:1056B000380200B200F01BF8182000F00EF805FBCD
:1056C000164000B200E006E000F011F8BDE8F04737
:1056D0005E2001F0A8BABDE8F08710B504465E2050
:1056E00001F0A1FA2046BDE8104001F09CBA10B5C7
:1056F0000446C0B201F097FAC4F30720BDE8104099
:1057000001F091BAC4010020A0860100240300200A
:1057100004050020040200201601002000007A4445
:10572000EC0000205801002070B52B4E90B03046A0
:1057300002F058F929480090294801A900240125C0
:1057400031C128020494CDE9054080000790202053
:1057500008900002CDE909046946304602F0AFF92D
:105760000121304602F0C8F98DF830400B948DF8D5
:1057700031504FF46020CDE90D04184C8DF83C50A9
:105780004C3C0BA9204602F099F803230122042186
:10579000204602F0E8F80121204602F0B8F8012185
:1057A000204602F0AAF8204602F0BBF8204602F09C
:1057B000BDF80028FAD1204602F0BFF8204602F0DA
:1057C000C1F80028FAD10121204602F0C2F810B039
:1057D00070BD034800887047080002404C24014017
:1057E0002C03002070472DE9FC47DFF8489105465F
:1057F00099F80000C0B300263746B0463446641C12
:10580000E4B26B4608223221532000F071FC9DF86F
:1058100000009DF80110202C00EB012000B206448E
:105820009DF802009DF8031000EB012000B2074430
:105830009DF804009DF8051000EB012001B29DF8D1
:105840000700884400F07F0001D20028D7D196FBE2
:10585000F4F0288097FBF4F0688098FBF4F0A880BF
:1058600089F80140BDE8FC87FFE76B46062232213C
:10587000532000F03DFC9DF800009DF8011000EB66
:10588000012028809DF802009DF8031000EB012004
:1058900068809DF804009DF8051000EB0120A880A9
:1058A000E0E7244810B500784FF0080200284FF0D8
:1058B0002D014FF053000ED000F014FC0A223121CC
:1058C000532000F00FFC0C222C21532000F00AFC86
:1058D0009022382108E000F005FC0A2231215320F3
:1058E00000F000FC0A222C21532000F0FBFB12499F
:1058F00040F20910088010BD38B5054600200C465E
:105900008DF8000001466B460122532000F0F0FBA9
:1059100018B19DF80000E52801D0002038BD0549E8
:105920002878087005482060054860600548A06038
:10593000012038BD2E03002004020020A3580008D7
:10594000E7570008E557000810B54FF4804420469B
:1059500002F02CF9012805D1204602F035F9B049B2
:105960000120087010BD30B4AD4AAE48918843891B
:10597000B0F91440C91A03895943C913B0F9123058
:105980000C44DB0293FBF4F31944C161906830BC12
:1059900000F0C7B838B5A24C207810B96088401C18
:1059A00060806B460322F621772000F0A1FB9DF872
:1059B00000009DF80110000440EA01209DF802104B
:1059C00008439849B1F92010C1F10801C840A0600E
:1059D00038BD94483421008C01EB80109049C2B24C
:1059E00000200870F421772000F07CBB38B58C4C87
:1059F000207810B96088401C60806B460222F62136
:105A0000772000F075FBBDF8000040BAA08038BDDB
:105A1000834900202E220870F421772000F062BB19
:105A20002DE9F043DFF8F891044685B099F80100BC
:105A300018B1012005B0BDE8F0834FF40058ADF86F
:105A40000C8002208DF80E001020774E8DF80F008C
:105A5000454603A9304602F00FFD4FF48047ADF8EC
:105A60000C7004208DF80F0003A9304602F004FDED
:105A700035610E21022002F08DFD00208DF8080016
:105A8000082001978DF8090001278DF80A7001A8F8
:105A900002F056F828208DF810000F208DF8110024
:105AA0008DF812008DF8137004A801F0D4FE1420B4
:105AB00000F012FF6B460122D021772000F018FB86
:105AC000584D9DF800000321E8752984552803D01E
:105AD000C6F814800020ADE76B460122D121772063
:105AE00000F006FB9DF8000000F00F012976000988
:105AF000687600F05EF889F8017041F2F8102080B5
:105B000046F29050608041F28830A0804748A06003
:105B10004748E06047482061474860614748A061C6
:105B200087E770B53F49CA69B1F90E30A2F57A62CC
:105B300002FB02F634136343DC12B1F90230534323
:105B400004EBE323B1F9004003EB84030C8CA34086
:105B50009B1C9D10B1F90430361353435A13B1F90D
:105B60000C30C988734302EB2342921C921002F559
:105B700000425143C90B401B4CF25032E2405043AB
:105B8000B0F1004F03D24000B0FBF1F002E0B0FBF7
:105B9000F1F040000112494340F6DE325143284AF9
:105BA0000914424301EB224101F6CF6100EB2110C1
:105BB00070BD00B587B06B461622AA21772000F091
:105BC00097FABDF8000041BA16480180BDF80210EE
:105BD00049BA4180BDF8041049BA8180BDF8061069
:105BE00049BAC180BDF8081049BA0181BDF80A1050
:105BF00049BA4181BDF80C1049BA8181BDF80E1037
:105C000049BAC181BDF8101049BA0182BDF812101D
:105C100049BA4182BDF8141049BA818207B000BD6B
:105C200030030020CC0A002000100140115A000867
:105C3000ED590008D3590008955900086759000824
:105C400043E3FFFF08B500208DF800006B460122FA
:105C50000A211E2000F04CFA18B19DF800004828D7
:105C600001D0002008BD012008BD08B54FF48050C8
:105C7000ADF8000002208DF8020004208DF803002A
:105C80006946264802F0F8FB642000F025FE7822E1
:105C900000211E2000F026FA322000F01DFE08BD73
:105CA00010B50446792200211E2000F01BFA322094
:105CB00000F012FE224601211E2000F013FA0122FC
:105CC0000221BDE810401E2000F00CBA10B5782269
:105CD00000211E2000F006FA202201211E2000F0E3
:105CE00001FA00220221BDE810401E2000F0FAB99E
:105CF0001CB504466B46062203211E2000F0F8F96D
:105D0000BDF8000040BA2080BDF8020040BA6080B3
:105D1000BDF8040040BAA0801CBD0000000C01408A
:105D200030B587B005464FF44060ADF8140002204E
:105D30008DF816001C208DF8170005A9FE4802F00A
:105D40009BFBFE4CE56000F014FAE06801F042FFB6
:105D5000684601F0AAFF00224FF44071E06801F0AC
:105D6000DAFF0025ADF804504BF6FF70ADF80600E1
:105D70004FF48040ADF80C00F14800900121E0683C
:105D800001F0A1FF6946E06801F037FF4FF4A06021
:105D900001F05CFD22208DF810008DF811508DF877
:105DA000125001208DF8130004A801F054FD2120A9
:105DB0008DF810008DF8115004A801F04CFD07B0CB
:105DC00030BD70B5DD4CE068858A15F4706F01D088
:105DD0000121217015F4E06F24D0018B00224FF4D3
:105DE000806101F098FFA8051CD4E068018889054E
:105DF00018D40188C9050CD50188C905FCD4012136
:105E000001F075FFE06801888905FCD4FFF788FF81
:105E100008E0012101F06BFF00224FF44071E068BF
:105E200001F079FFE068818A21F4706181820020AD
:105E3000207170BDC5E72DE9F041C04CE068818A52
:105E40004FF00105C9B2CA074FF0000627D00188FC
:105E500021F400610180012101F053FFE670607AB6
:105E600020B1607860B9A079FF2809D0617900225B
:105E7000E06801F05DFFA079FF280FD0FF20B8E0B7
:105E80006570E079022804D1E068018841F400617E
:105E9000018061790122E06801F04AFFC9E08A07C8
:105EA0004FF4806734D5BFF3508FE079012810D1CB
:105EB000607A70B1607860B10021E06801F021FF84
:105EC000BFF3508FE068018B012101F010FFA57036
:105ED0001CE0E068008BBFF3508FE07902280DD101
:105EE000607A58B1607848B10021E06801F009FF9C
:105EF00093E03946E06801F00EFF9AE0E07903286C
:105F000004D1607A10B16078002874D10122F0E7E2
:105F10004A0753D5A570627A88494978CAB3C9B38C
:105F2000E17902291FD9002101F0EBFEE06801F0C0
:105F3000FCFE94F9032063699854521CE27001211D
:105F4000E06801F0D4FEA570E06801F0EEFE94F97F
:105F5000031062695054491CE17001223946E0681F
:105F600001F0D9FE25E0012101F0C1FEE06801F059
:105F7000DCFE94F9031062695054491CE170E0683A
:105F800001F0D3FE94F9031062695054891CE1704A
:105F90000FE000E000E009B9217A31B1012101F000
:105FA000A6FEE078401CE07003E0012101F095FEC0
:105FB0006570E0680188C905FCD43AE04A061BD543
:105FC00001F0B3FE94F9031062695054491C48B2C1
:105FD000E070E179C01C814204D100223946E068BA
:105FE00001F099FEE17994F90300814221D100F199
:105FF0000100E0701DE010E009061AD594F90320B5
:10600000511C4BB20BD02569A95CE37001F08BFEEB
:10601000E07994F9031088420BD1002269E7E3701C
:10602000A17901F080FE607A0028F6D1E07900289D
:10603000F3D094F90310E079401C814209D16670D5
:10604000A07828B100224FF44071E06801F063FEAF
:106050002671BDE8F081EEE6B3E6ECE67FB5374C9D
:10606000400047F230556071A17101212172002674
:106070006672C4F810D0C4F814D06846E271217179
:106080002670102A02D9002004B070BD002103E060
:106090005E5C4654491CC9B29142F9D3E0688188DC
:1060A00089050ED40188C90505D401888905FCD469
:1060B000012101F012FE01224FF44071E06801F06D
:1060C0002AFE207910B16D1EFBD104E01DB12078AD
:1060D00080F00100D8E76089401C6081E068FFF72C
:1060E0001FFED0E707B502AB0122FFF7B7FF0EBDD9
:1060F00070B5124C4FEA400047F230556071A17103
:10610000002020720121617263612361E2712171BB
:106110002070E0688188890516D40188C90505D4F6
:1061200001888905FCD4012101F0D7FD01224FF43B
:106130004071E06806E00000000C01403C030020D4
:10614000801A060001F0E7FD207910B16D1EFBD129
:1061500004E01DB1207880F0010070BD6089401C12
:106160006081E068FFF7DCFD002070BD2F484089AA
:1061700070472DE9F8434FF44067ADF800704FF0D9
:1061800002088DF802801420294C8DF8030069461E
:10619000204602F071F93946204602F0CEF900257A
:1061A000261502E00A2000F08CFB3146204602F062
:1061B000BDF90028F6D03146204602F0C0F90A2089
:1061C00000F07FFB3146204602F0B7F90A2000F0CC
:1061D00078FB6D1CEDB2082DE7D34FF4006529461E
:1061E000204602F0ACF90A2000F06BFB3146204655
:1061F00002F0A5F90A2000F064FB3146204602F0C7
:106200009CF90A2000F05DFB2946204602F095F932
:10621000ADF800708DF802801C208DF803006946EF
:10622000204602F029F9BDE8F88300003C03002075
:10623000000C014038B504466B4602221B21682041
:10624000FFF756FFBDF8000043F2903140BA084412
:106250004FF48C71B0FBF1F02330208038BDB0F9E1
:106260000010CA1701EB927189100180B0F9021079
:10627000CA1701EB927189104180B0F904104942AC
:10628000CA1701EB92718910818070471CB50446D2
:106290006B4606221D216820FFF72AFFBDF800008B
:1062A00040BA2080BDF8020040BA6080BDF804000A
:1062B00040BAA0801CBD10B5192000F00DFB0022D3
:1062C00015216820FFF70EFF10B9032000F089FBAD
:1062D00028481621007840F018026820FFF702FFD6
:1062E000002217216820FFF7FDFE01223D216820D2
:1062F000FFF7F8FE01223E21BDE810406820FFF7BD
:10630000F1BE10B50446192000F0E6FA002215216E
:106310006820FFF7E7FE002808D0174820601748DC
:1063200060601748A0601748E060012010BD114967
:10633000622817D006DC0A281AD0142816D02A287A
:1063400009D111E0BC2804D0B0F5807F03D1002032
:1063500000E0012008700878162140F0180268203B
:10636000FFF7C0BE0220F5E70320F3E70420F1E7C2
:106370000520EFE754030020B76200088D62000893
:106380005F620008356200083EB505460C46684667
:1063900001F074FFF848641EADF804400068F74946
:1063A000B0FBF1F0401EADF800000020ADF8060093
:1063B000ADF802006946284601F040FD3EBD70B5CB
:1063C0001646EF4B00EB800203EB8205ED4A02EB31
:1063D00000142068FFF7D8FFD4E90101002200F083
:1063E0003CFA217B3246206800F0DCF9A07B18B132
:1063F0000121206801F067FF0121206801F059FFA9
:10640000207B30B1042807D008280AD00C2806D1F8
:106410000AE02068343001E020683830686028469F
:1064200070BD20683C30F9E720684030F6E7F8B5E9
:1064300017460E46D24A00EB800102EB8105D14996
:1064400001EB00144FF6FF712068FFF79DFFD4E9C0
:106450000101012200F001FA217B0022206800F0F6
:10646000E4F90121206801F024FF607B8DF8000031
:1064700000208DF8010001208DF802008DF8030046
:10648000684601F0E8F92E60AF72207B30B1042835
:1064900008D008280DD00C2809D10EE001220221D5
:1064A000206802E001220421206801F017FF28463D
:1064B000F8BD012208212068F7E701221021206899
:1064C000F3E770B5B04C0221204601F032FFAC4D2D
:1064D000012814D01021204601F02BFF01281AD1E9
:1064E00009261021204601F02FFF204601F01EFF53
:1064F000D5F8B42001463046BDE870401047082664
:106500000221204601F020FF204601F009FF01464C
:10651000D5F8A020EFE770BD70B50C460646022105
:1065200001F007FF964D012823D00421304601F0E9
:1065300000FF012826D00821304601F0FAFE01288C
:106540002AD01021304601F0F4FE01282ED1E41C9F
:1065500064B21021304601F0F7FE304601F0E6FE4D
:10656000014604EB840055F82020E0B2BDE87040FD
:10657000104764B20221304601F0E6FE304601F0D9
:10658000CFFEEDE7641C64B20421304601F0DCFE6E
:10659000304601F0C7FEE3E7A41C64B20821304690
:1065A00001F0D2FE304601F0BFFED9E770BD0021F8
:1065B0004FF08040B0E704217448ADE70A217448E9
:1065C000AAE7704A30B5083A00239088D0809180BD
:1065D000081A81B240F68C20814201D9D37030BDB7
:1065E0006848A1F2EF24083840F2DB55C078AC428D
:1065F00004D2082802D2674C24F81010401CD07036
:106600006548038030BD5E4A00EB800370B502EB45
:1066100083025C4BD47A03EB001318681B7B84B1B4
:10662000D18194895B4D091B1182947A25F814104D
:106630000024D4722246194600F0F7F85648048028
:1066400070BD91810121D172BDE8704002221946CE
:1066500000F0EBB82DE9F04704460020617901B164
:106660000220617801B1401C4649DFF81081E03119
:10667000002551F82070A1F1E8064FF47A797A5D8F
:1066800002F00F0002F0F001FF2A56D0A2781AB1F2
:1066900002284FD003284DD011F0300F02D02278BD
:1066A00002B90021E27832B1627922B9082801D01A
:1066B000092800D1802122792AB162791AB9021FF2
:1066C000032A00D88021CA0605D500223349FFF7E6
:1066D000AEFE082008E08A0608D5B2783049FFF7F8
:1066E000A6FEB07800F10100B07023E04A0610D594
:1066F000E288B8FBF2F189B24A46FFF760FE014634
:10670000244A3078103242F8201000F10100307035
:1067100010E009060ED52289B8FBF2F189B24A468B
:10672000FFF74DFE01461B4A7078403242F82010B8
:10673000401C70706D1C0E2DA1DB0020BDE8F087A1
:10674000104A083A1278904205D2124A103252F892
:1067500020004068018070470A4A083A5278904207
:1067600005D20C4A403252F8200040680180704740
:10677000084931F810007047A004002040420F0083
:10678000F00A002060030020002C014000040040BB
:1067900000080040080C002048010020C3650008E4
:1067A000076600087FB506460C461546684601F0A8
:1067B0006EFD7020ADF800000120ADF80200002051
:1067C000ADF804000220ADF80800C001ADF8065095
:1067D000ADF80C0074B1042C15D0082C1CD00C2C76
:1067E00007D16946304601F009FC0821304601F026
:1067F00090FD7FBD6946304601F059FB08213046C7
:1068000001F074FD7FBD6946304601F085FB08212B
:10681000304601F071FD7FBD6946304601F0B6FBA0
:106820000821304601F06FFD7FBDFEB506460C46DF
:106830001546684601F035FD0120ADF80400002141
:10684000ADF80040ADF80610ADF80810ADF80250F4
:106850006946304601F07AFCFEBDF8B506460C46A6
:106860001546684601F05AFEADF800400DB12820EB
:1068700000E018208DF8030002208DF80200694620
:10688000304601F0F9FDF8BD6C484168491C416093
:10689000704710B569494FF0E02348689A694C6821
:1068A000A042FAD16649891A4822B1FBF2F100EB05
:1068B0004002C2EBC01001EBC00010BD5F48406851
:1068C000704730B50546FFF7E4FF0446FFF7E1FFE8
:1068D000001BA842FAD330BD30B504464FF47A7598
:1068E00002E02846FFF7EDFF641EFAD230BD2DE925
:1068F000F0418CB01822534901A802F060F8032738
:1069000000F0C0FE0121504801F077FA012144F661
:106910001D2001F069FA0121084601F05CFA01F03E
:106920007EFA4FF6FF70ADF8000000268DF8036088
:106930006946464801F0A0FD6946454801F09CFDC6
:106940006946444801F098FD0121434801F0F9FDF2
:10695000002401AD4FF0020805EBC4008188ADF8BA
:1069600000108DF8028080798DF8030055F834000E
:10697000694601F081FD641CBC42EDD33448082116
:10698000103001601021016030498014103108601E
:1069900007A801F0DBF931490798B0FBF1F027496E
:1069A00008602F484FF47A710068B0FBF1F0B0F145
:1069B000807F0BD220F07F414FF0E020491E4161E3
:1069C000284AF0211170866107210161FEF7ACFEB3
:1069D0002548FFF7A5F96420FFF77EFF0CB0BDE85E
:1069E000F0811B4A1021143211600821121F11601E
:1069F000044640F2DB10154F151F44434E02143776
:106A0000A7F1040C286880F010002860286880F046
:106A100008002860A01EFFF75FFF3E601920FFF707
:106A20005BFFCCF80060EDE710B111490F4808603A
:106A30000C491048173908607047000050040020C6
:106A40004019010078B60008070040000008014026
:106A5000000C0140001001400002300040420F00D5
:106A6000A004002023ED00E000580040EFBEADDEA2
:106A7000F04F00200400FA05CD48CC4A8168531835
:106A8000CC4A1365C3688B4203D9591A9164836059
:106A900004E0C1F58071916400218160C548012145
:106AA000443001F029B810B54FF4005001F03AF825
:106AB000C0480021443001F01FF8BD48083003C829
:106AC000814202D0BDE81040D6E710BD2DE9F0416B
:106AD00092B004464FF40070ADF83C0002208DF8EF
:106AE0003E001820B44D8DF83F000FA9284601F054
:106AF000C3FC2815ADF83C0048208DF83F000FA9D5
:106B0000284601F0B9FC0E208DF8400001218DF8D7
:106B100041108DF842108DF8431010A800F09BFE34
:106B20000B940024ADF834400C20DFF89082ADF8CF
:106B30003040ADF83600ADF83240ADF838400BA922
:106B4000404601F005FC9B4F5837384600F04AFF9D
:106B5000A81408F104050095CDE909049848CDE989
:106B6000010480260494CDE90564A8150390202033
:106B7000CDE907406946384600F0A1FF01213846BB
:106B800000F0BAFF01224021404601F066FC384681
:106B900000F0C5FF8649874F44374860384600F00B
:106BA00021FF1020029000950494CDE9056407941C
:106BB00069463846089400F082FF012202213846D7
:106BC00000F0A5FF7B48846401228021404601F04B
:106BD00044FC0121404601F01EFC12B0BDE8F081EA
:106BE000744810B5583000F09AFF714949688842DE
:106BF00001D0012010BD002010BD6D48D0E9021069
:106C0000814201D1012070470020704768496C4BD8
:106C10004A68C2F58070185C521E4A6002D14FF477
:106C200080724A607047624A604BD1685854491C70
:106C3000C8B2D0605F48406CC00700D11CE7704705
:106C400010B5044602E0641CFFF7EDFF2078002831
:106C5000F9D110BD1FB50446684601F0D1FB0020F4
:106C60005349ADF804000094ADF80600ADF80800F3
:106C7000097809B1002100E0082141F00401514CDC
:106C8000ADF80A10ADF80C006946204601F060FB33
:106C90000121204601F0BFFB1FBD2DE9FC410F463D
:106CA000804601211446480401F0A7F8404D2620F3
:106CB00002262C708DF8040001208DF805008DF857
:106CC00006608DF8070001A800F0C5FD0420ADF8AE
:106CD00000008DF802601820374E8DF803001CB9B3
:106CE0006946304601F0C8FB0820ADF80000482096
:106CF0008DF803006946304601F0BEFB4046FFF7C1
:106D0000A9FF304E012240F22551304601F08DFBA3
:106D10002CB9012240F22771304601F086FB2F6129
:106D2000BDE8FC8196E722490A78002A0CD1264B5F
:106D30008A699854521C02F07F008861012240F257
:106D40002771204801F071BB70471948D0E9051040
:106D5000814201D1012070470020704770B5194E63
:106D6000358840F22550124C054206D0206920B1EA
:106D7000304601F07AFB2169884728060CD5D4E912
:106D80000510814209D01048405C0E4A121D108047
:106D9000491C01F07F00606170BD3046BDE8704065
:106DA000002240F2277101F040BB0000680D002076
:106DB0005804002000000240000801400038014053
:106DC000680C002000440040680E0020FEB5384CDE
:106DD0000125207878B1012822D002281FD1642013
:106DE0008DF8000033488DF8015000264078A0B39C
:106DF0008DF8025043E07A208DF800002E486B4653
:106E00000222B0F90000FF21C0F1B40000EBD07005
:106E100040108DF801006D20FFF720F92570FEBDB0
:106E2000264979208DF80000B1F900000A2290FB74
:106E3000F2F010F15A0301D5002003E05A30B428D3
:106E400000DDB4208DF80100B1F9020090FBF2F0F2
:106E500010F15A0102D5002004E00EE05A30B428A7
:106E600000DDB4208DF802006B460322FF216D2067
:106E7000FFF7F4F802202070FEBD8DF802606B462B
:106E80000322FF216D20FFF7E9F82670FEBD08B54B
:106E90006B208DF800000A208DF801008DF80200AB
:106EA0006B460322FF216D20FFF7D8F808BD0000D4
:106EB000740400208C08002044020020CC00002034
:106EC000B0F90010CA1701EB927189100180B0F976
:106ED0000210CA1701EB927189104180B0F90410B9
:106EE0004942CA1701EB92718910818070471CB525
:106EF00004466B46062243216820FFF7F9F8BDF8E7
:106F0000000040BA2080BDF8020040BA6080BDF8A1
:106F1000040040BAA0801CBD08B54FF40050ADF885
:106F2000000002208DF8020004208DF8030069465D
:106F30004C4801F0A1FA80226B216820FFF7D2F8BB
:106F40000520FFF7C9FC002219216820FFF7CAF8C5
:106F500003226B216820FFF7C5F802223721682041
:106F6000FFF7C0F803221A216820FFF7BBF81822A8
:106F70001B216820FFF7B6F83B48007814280BD097
:106F8000152809D0542807D0552805D010221C21D7
:106F90006820FFF7A7F808BD0822F8E7B0F902104B
:106FA000B0F90020CB1701EB5371C9100180514299
:106FB000CA1701EB5271C9104180B0F90410CA1709
:106FC00001EB5271C910818070471CB504466B46B5
:106FD00006223B216820FFF78BF8BDF8000040BA7D
:106FE0002080BDF8020040BA6080BDF8040040BABD
:106FF000A0801CBD1D4940F2FF3008807047F8B5E5
:1070000004460D4616462320FFF766FC6B46012218
:1070100075216820FFF76CF8002808D09DF8000063
:1070200000F07E008DF80000682801D00020F8BD37
:107030001EB10D495520087005E00B4B01220C21B3
:107040006820FFF755F80A4820600A4860600A483F
:10705000A0600A4828600A4868600A48A8600120C1
:10706000F8BD0000000C014075040020040200205F
:10707000F56F0008CB6F00089D6F0008196F0008BE
:10708000EF6E0008C16E0008B0F900104942CA173F
:1070900001EB927189100180B0F902104942CA17C0
:1070A00001EB927189104180B0F90410CA1701EB0D
:1070B00092718910818070471CB504466B46062288
:1070C00001211C20FFF714F8BDF8000040BA00B2FF
:1070D0002080BDF80210801049BA09B26180BDF865
:1070E0000420208052BA881012B260809010A080D4
:1070F0001CBD08B52020ADF8000002208DF802006C
:1071000004208DF803006946264801F0B5F90022F5
:107110002A211C20FEF7E6FF02220E211C20FEF78A
:10712000E1FF03220F211C20FEF7DCFF12222B219E
:107130001C20FEF7D7FF02222C211C20FEF7D2FFD5
:1071400001222D211C20FEF7CDFF00222E211C2024
:10715000FEF7C8FF05222A211C20FEF7C3FF1249B3
:107160004FF48070088008BD38B5044600208DF8C3
:1071700000006B4601220D211C20FEF7B9FF28B14B
:107180009DF800002A2803D01A2801D0002038BD1D
:1071900006492160064961600649A16006490870F8
:1071A000012038BD0008014004020020F3700008EF
:1071B000B9700008897000087604002010B5444CAE
:1071C0004448A18801F0B2F918B1FFF762FBA06052
:1071D0000AE0FFF75EFBA168884205D9401A3B210F
:1071E00090FBF1F061690880E068BDE8104000F0B4
:1071F000EBBCE3E7E2E7FEB50125354C022110B117
:10720000012810D109E04FF4807060804000A08018
:10721000E06009202070172004E06580A180E16013
:107220002570072060706088ADF8000010268DF88A
:107230000360284F8DF802106946384601F01CF9AA
:10724000A088ADF8000004208DF803006946384698
:1072500001F012F92178012001F09CF9E06800F0BA
:10726000B3FCE068019000208DF808008DF80960FB
:107270008DF80A5001A800F063FC94F9010000F0B9
:107280001F018D4040094FF0E02101EB8000C0F864
:107290000051FFF713FB3C382061FEBD70B5054679
:1072A000FFF70CFB0A4C21693C3188420FD3C4E93B
:1072B0000405084D6188284601F03FF90B20FFF7CF
:1072C00000FB61882846BDE8704001F038B970BD08
:1072D00078040020000C0140B0F900104942CA17A0
:1072E00001EB927189100180B0F90210CA1701EB0D
:1072F000927189104180B0F904104942CA1701EB1C
:1073000092718910818070471CB504466B46062235
:10731000A8216820FEF7ECFEBDF8000040BA6080AE
:10732000BDF8020040BA2080BDF8040040BAA08039
:107330001CBD10B56420FFF7CFFAF022232168208E
:10734000FEF7D0FE10B90320FFF74BFB0520FFF737
:10735000C3FA1E4820210078BDE8104040F00F021B
:107360006820FEF7BFBE38B504461920FFF7B4FA0F
:107370006B4601220F216820FEF7BAFE9DF800003F
:10738000D32801D0002038BD11482060114860602A
:107390001148A060012038BD0C49202806D03628AD
:1073A00006D04E280DD05D2804D10CE0002000E06E
:1073B000402008700878202140F00F026820FEF776
:1073C00091BE8020F5E7C020F3E700009004002084
:1073D0003373000809730008D97200082DE9F04FD3
:1073E000DFF87CA2DFF87CE24FF00008BAF80A1060
:1073F000DEF80400BAF80830A0EB0122A3FB026714
:10740000BAF80400D517040408FB027003FB050357
:10741000F00940EA436014EB000BBAF80640BAF8F2
:107420000200A4FB027C4FEAC03548EBE311404662
:1074300000FB02C34FEAE27604FB06334FEA17244F
:1074400044EA036415EB040C40EB2320BAF80C303B
:107450004446A3FB02674FEAE27504FB027203FB9A
:1074600005224FEA422343EAD6524FF4FA63D21878
:10747000C146B2F5FA6F17DAA2F5FA635B4303EB84
:1074800083034FEA63084FEAA309774B9A420BDA6A
:1074900002F2DC525243C2EBC203984402EB4203B5
:1074A00003EBC20309EB6309BBEB080261EBE87174
:1074B000BCEB0903DEF808404FF00005A4FB0367AE
:1074C00005FB037360EBE97004FB00304FEA565391
:1074D00043EAC0234FEA60509A1A60EB010041046E
:1074E00041EAD230BDE8F08F10B500F070F85D4988
:1074F000886010BD5B48012200784030C1B277201F
:10750000FEF7F0BD10B500F062F85649486010BDB6
:107510005448012200785030C1B27720FEF7E2BD16
:107520002DE9FE4305464FF40054ADF8004002201B
:107530008DF8020010204D4E8DF80300694630464C
:1075400000F09AFF74610A20FFF7C6F902AB01222E
:10755000A0217720FEF7CCFD002823D001221E2198
:107560007720FEF7BFFD4FF42F60FFF7AAF9002444
:10757000DFF8EC802646A02707EB4400C1B201AB40
:10758000022277200196FEF7B3FDBDF8040040BA51
:1075900028F81400641C082CEEDB314800F029F8B0
:1075A00010B10020BDE8FE8342F210702880688090
:1075B0004FF47A60A8802E48A8602E48E8602E48D4
:1075C00028612E4868612E48A8610120EAE708B5C5
:1075D0006B46032200217720FEF78AFD9DF800000C
:1075E0009DF80110000440EA01209DF802100843B4
:1075F00008BDF0B5C289002102F47F4502F00F04F6
:107600000123C5814FEA010230F8126006B1002360
:10761000521C082AF8DB4FF0FF36F3B90022D307DB
:1076200022F00103C35A02D0DBB2594001E081EAE3
:10763000132108230F0401D581F4C05149005B1EBA
:10764000002BF7DC521C102AE9DB2543C581C1F36E
:107650000330844201D10020F0BD3046F0BD00006F
:10766000E80E00209404002024FAFFFF00100140DF
:107670001175000805750008F5740008E974000824
:10768000DD730008694A10B55068694910F00C03B1
:10769000684803D0042B01D0082B0BD0016051683F
:1076A000644AC1F30311121D515C026822FA01F20F
:1076B000026010BD5168536801F470114FF002046C
:1076C00013F4803F04EB914102D053689B0301D532
:1076D000594B00E0564B5943E0E7544810B4026858
:1076E000002142F4803202604FF4A063026801F18D
:1076F000010112F4003F01D19942F7D101688A03D8
:107700004E4931D50A6842F010020A600A6822F038
:1077100003020A600A6842F002020A60416841609E
:1077200041684160416841F480614160416821F4F1
:107730007C114160416841F4E8114160016841F009
:107740008071016001688901FCD5416821F0030165
:107750004160416841F0020141604168C1F381012B
:107760000229FAD110BC7047026842F0010202609F
:107770000022046802F1010214F0020F01D19A42C2
:10778000F7D102689207EDD50A6842F010020A604C
:107790000A6822F003020A600A6842F002020A60E4
:1077A0004168416041684160416841F480614160E5
:1077B000416821F47C114160416841F460114160ED
:1077C000016841F08071016001688901FCD5416860
:1077D00021F003014160416841F0020141604168CC
:1077E000C1F381010229FAD110BC4BE70F4810B553
:1077F000016841F0010101604168114A1140416096
:107800000168104A11400160016821F48021016083
:10781000416821F4FE0141604FF41F018160FFF7D0
:107820005CFF09494FF00060086010BD0010024085
:1078300000127A00A004002000093D000020024050
:107840000000FFF8FFFFF6FE08ED00E018490843CE
:1078500018490860704770B50F21C4780278012379
:107860004FF0E026DCB1134C246804F4E064C4F566
:10787000E064250AC5F10404E9404578A540847810
:107880000C402C4321010C4C1155007800F01F01D5
:107890008B40400906EB8000C0F8003170BD02F05B
:1078A0001F008340500906EB8000C0F8803170BD96
:1078B0000000FA050CED00E000E400E010B54268BD
:1078C000464B0C791A400B6842EA0422134343608A
:1078D0008368434A1340D1E9024222434C7943EA88
:1078E00044031A438260C26A097C22F47002491E72
:1078F000C9B242EA0151C16210BD0029816802D0BB
:1079000041F0010101E021F001018160704700298F
:10791000816802D041F4807101E021F480718160BE
:107920007047816841F0080181607047014600207E
:107930008968090700D501207047816841F004017A
:1079400081607047014600208968490700D5012001
:1079500070470029816802D041F4A00101E021F4C0
:10796000A0018160704770B5072509290AD9C4684C
:10797000A1F10A0606EB4606B540AC43B3401C43F2
:10798000C46007E0046901EB4106B540AC43B34075
:107990001C4304611F23072A09D2446B521E02EBC9
:1079A000820293409C4391400C43446370BD0D2A76
:1079B00009D2046BD21F02EB820293409C43914098
:1079C0000C43046370BDC46A0D3A02EB820293401B
:1079D0009C4391400C43C46270BD0000FFFEF0FF69
:1079E000FDF7F1FF01684FF6FE72114001600021C2
:1079F000016041608160C1604F494F4A083990423F
:107A000003D1486840F00F0006E04B4A1432904220
:107A100004D1486840F0F00048607047464A283278
:107A2000904203D1486840F47060F5E7424A3C3226
:107A3000904203D1486840F47040EDE73E4A50322E
:107A4000904203D1486840F47020E5E73A4A643236
:107A5000904203D1486840F47000DDE7364A78323E
:107A6000904203D1486840F07060D5E7334A111F57
:107A7000904203D1086840F00F0006E02F4A14320C
:107A8000904204D1086840F0F000086070472B4A2B
:107A90002832904203D1086840F47060F5E7274A25
:107AA0003C32904203D1086840F47040EDE7234A2D
:107AB00050329042EAD1086840F47020E5E730B5D2
:107AC000036847F6F07293430C6A8A682243D1E94F
:107AD00004452C4322438C692243CC6922434C6ADF
:107AE00022438C6A22431A430260CA6842600A68D1
:107AF00082604968C16030BD0029016802D041F050
:107B0000010102E04FF6FE72114001607047002A49
:107B1000026801D00A4300E08A430260704740686F
:107B200080B27047C10003D50449091F086070473F
:107B300001490839486070470800024008040240C3
:107B400030B523498379026853B30B6893430B60C4
:107B50000A1D13680468A343136002790A4413687A
:107B60000468234313601A4A083213680468A34365
:107B70001360131D1C680568AC431C604479102C0D
:107B800005D021440A68006802430A6030BD1168CC
:107B9000046821431160196800680143196030BD11
:107BA0000079084401689143016030BD084A0146EC
:107BB00000201268064B0A4014331B680B4202D0A7
:107BC000002A00D001207047014914310860704735
:107BD000000401405A4910B588424FF0010101D11B
:107BE0004C0501E04FF48004204600F00FF92046D8
:107BF000BDE81040002100F009B970B50446808846
:107C000086B00D4620F03F06684600F09FF84D49CB
:107C10000298B0FBF1F189B20E43A680228822F0CF
:107C200001022280484B2A689A421CD85200B0FBBD
:107C3000F2F080B2042800D20420491C2184A083E1
:107C4000208840F00100208021884FF6F530014067
:107C5000A8886A89104308432080A8892989084395
:107C6000208106B070BDEB88A3F53F46FF3E05D1ED
:107C700002EB4202B0FBF2F080B208E002EBC2037A
:107C800003EB0212B0FBF2F080B240F48040020538
:107C900001D140F001004FF4967251434FF47A72D3
:107CA000B1FBF2F140F40040C7E741F288310160D6
:107CB000002181804BF6FF72C280018141814FF427
:107CC0008041818170470029018802D041F0010183
:107CD00001E021F00101018070470029018802D0F4
:107CE00041F4807101E021F4807101807047002926
:107CF000018802D041F4007101E021F4007101809B
:107D000070470029018802D041F4806101E021F42C
:107D1000806101807047002A828801D00A4300E018
:107D20008A438280704701827047008AC0B27047E0
:107D300012B141F0010101E001F0FE010182704742
:107D40000054004040420F00A0860100374910B5A2
:107D50004A6812F00C03364A03D0042B01D0082BDA
:107D600026D002604A68334B02F0F00212099C5C94
:107D70000268E24042604C6804F4E064240A1C5D3E
:107D800022FA04F484604C6804F460544FEAD4246A
:107D90001B5D22FA03F2C2604968264B01F44041A0
:107DA0004FEA91311B1F595CB2FBF1F1016110BD2B
:107DB0004A684B6802F470124FF0020413F4803FDB
:107DC00004EB924202D04B689B0301D51A4B00E0B2
:107DD000174B5A43C5E7154A0029516901D00143A1
:107DE00000E0814351617047104A0029916901D038
:107DF000014300E08143916170470C4A0029D16939
:107E000001D0014300E08143D1617047074A002956
:107E1000116901D0014300E08143116170470348BB
:107E2000416A41F0807141627047000000100240D9
:107E300000127A00B804002000093D0030B5028825
:107E4000F84BF94C98420DD0A0420BD0B0F1804FC6
:107E500008D0F64DA84205D0F54DA84202D0F54D08
:107E6000A84203D122F070054A882A43F24DA84265
:107E700006D0F24DA84203D022F44075CA882A43A6
:107E800002808A8882850A88028598420AD0A042A8
:107E900008D0EB4A904205D0EA4A904202D0EA4A22
:107EA000904201D1097A01860121818230BD30B52D
:107EB000028C22F001020284028C8388048B22F05F
:107EC000020224F073050C882C430D8915434A885F
:107ED0002A43D44DA8420BD0D34DA84208D0D84D48
:107EE000A84205D0D74DA84202D0D74DA8420DD107
:107EF00022F008054A8923F440732A4322F004053E
:107F00008A882A438D891D43CB892B438380048330
:107F1000C9888186028430BD30B5028C22F01002FF
:107F20000284028C8388048B22F0200224F4E6452C
:107F30000C88240645EA14440D892D0542EA1545AE
:107F40004A88120545EA1242B64DA84202D0B64D03
:107F5000A84215D122F080054A8923F44063120516
:107F600045EA124222F040058A88120545EA12428B
:107F70008D89AD0443EA1545CB899B0445EA13433B
:107F800083800483C9880187028430BD30B5028CA8
:107F900022F480720284028C8388848B22F4007223
:107FA00024F073050C882C430D892D0642EA1545F3
:107FB0004A88120645EA12429A4DA84202D09A4DCA
:107FC000A84215D122F400654A8923F440531206D1
:107FD00045EA124222F480658A88120645EA124276
:107FE0008D892D0543EA1545CB891B0545EA1343C9
:107FF00083808483C9888187028430BD30B5028C38
:1080000022F480520284038C8288848B24F4E64517
:108010000C88240645EA144423F400550B891B07F9
:1080200045EA13434D882D0743EA15457D4B984299
:1080300002D07D4B984205D122F480438A89920573
:1080400043EA124282808483C988A0F840100584E4
:1080500030BD828B22F440628283828B42EA01220D
:1080600082837047828B22F00C028283828B0A43C8
:1080700082837047028B22F440620283028B42EAC1
:1080800001220283704770B5048C24F0100404842C
:10809000068B048C26F473461B0746EA134312062C
:1080A00043EA12420D055F4B2D0C98420ED05E4BF9
:1080B00098420BD0B0F1804F08D05C4B984205D06D
:1080C0005B4B984202D05B4B984205D124F02001D3
:1080D000294341F0100104E024F0A0030B4343F0D6
:1080E00010010283018470BD028B22F00C02028316
:1080F000028B0A430283704730B5048C24F00104DC
:108100000484058B048C1B0542EA134325F0F30518
:10811000444A2B4390420ED0434A90420BD0B0F1D8
:10812000804F08D0414A904205D0414A904202D047
:10813000404A904202D124F0020201E024F00A02F7
:108140000A4342F001010383018430BD2DE9F05F51
:108150000D4604460E883348DFF8CCC0DFF8CCA0CB
:10816000DFF8CCE04988AA882B894FF0804B3EB3DA
:10817000042E2DD0082E268C32D026F4805626844C
:10818000B4F81C90268C0F074FEA1748120629F402
:1081900073471B0747EA124242EA134384420AD05C
:1081A000644508D05C4506D0544504D0744502D0DF
:1081B0002048844256D126F4005040EA080054E09A
:1081C0002046FFF799FFE9882046BDE8F05F8BE77E
:1081D0002046FFF758FFE9882046BDE8F05F49E7F1
:1081E00026F480762684A78B268C1B0527F0F307C0
:1081F00042EA13434FEA01683B434FEA184884427E
:108200000AD0644508D05C4506D0544504D0744576
:1082100002D00848844219D126F4007040EA0800D0
:1082200017E00000002C0140003401400004004031
:1082300000080040000C0040001000400014004006
:1082400000400140004401400048014026F4206005
:10825000084340F48070A3832084E9882046BDE869
:10826000F05FFFE626F40240084340F48050A38309
:108270002084E9882046BDE8F05FEAE64FF6FF710A
:10828000818000210180C1804180017270470021FE
:10829000018041808180C180018141818181C181D2
:1082A000704700210180418001228280C1800181CC
:1082B00070470029018802D041F0010101E021F05E
:1082C000010101807047002930F8441F02D041F4B9
:1082D000004101E0C1F30E0101807047002A82894C
:1082E00001D00A4300E08A4382817047028B22F06A
:1082F00008020A4302837047028B22F4006242EABA
:10830000012101837047828B22F008020A43828395
:108310007047828B22F4006242EA01218183704718
:10832000808E7047008F7047808F7047B0F8400094
:108330007047038A002280890B4200EA010001D0C5
:1083400000B1012210467047C94301827047000006
:1083500030B50446008A85B00D464CF6FF710840E2
:10836000E98801432182A1894EF6F3100140A888D3
:108370002A8910436A890A431043A081A08A4FF6D4
:10838000FF410840A9890143A1826846FFF7DEFC4E
:108390003848844201D1039800E00298A189090479
:1083A000002900EBC00101EB0010296802DA4FEA56
:1083B000410101E04FEA8101B0FBF1F06422B0FB22
:1083C000F2F14FEA01114FEA11136FF018056B43F8
:1083D00000EB8300A3891D044FF0320306D503EBA5
:1083E000C000B0FBF2F000F0070005E003EB001066
:1083F000B0FBF2F000F00F000843208105B030BD63
:108400004FF41651016000218180C18001810C224E
:108410004281818170470029818902D041F4005155
:1084200001E021F400518181704710B5C1F342137E
:1084300001F01F040121A140012B07D0022B07D01E
:108440001430002A026805D00A4304E00C30F8E733
:108450001030F6E78A43026010BD002A828A01D0FC
:108460000A4300E08A43828270478088C0F3080094
:1084700070470000003801402DE9F041CB7800251D
:1084800003F00F02DB0601D58B781A430B884FF0FF
:108490000F0813F0FF0F4FF0010C1CD0D0F8004074
:1084A0000E880CFA05F31E409E4210D1AF0008FA68
:1084B00007F624EA060602FA07F43443CE78282E9B
:1084C00002D0482E02D002E0436100E003616D1C3F
:1084D000082DE5D304600B88FF2B1DD944680025C7
:1084E00005F108060CFA06F30E881E409E420FD1D5
:1084F000AF0008FA07F624EA060602FA07F4344346
:10850000CE78282E00D14361CE78482E00D1036169
:108510006D1C082DE4D34460BDE8F0814FF6FF7177
:108520000180022181700421C17070470246002041
:1085300092680A4200D00120704701617047416192
:108540007047F0B51C4C002801DAE36900E063686D
:10855000420D120185B2C0F301579540C0F30346A6
:10856000032F05D0C2020AD50322B240934307E08D
:1085700023F07062636823F07063636002E0AB43D2
:1085800043F0706201B12A43002801DAE261F0BDD4
:108590006260F0BD10B58A0721F003040649130F8D
:1085A00021440F228C689A4094438C608A689840DA
:1085B00002438A6010BD0000000001403748364980
:1085C00041603749416070473448016941F080019A
:1085D0000161704731490420CA68D20701D00120E7
:1085E0007047CA68520701D502207047C968C9069A
:1085F000FBD50320704700B50346FFF7EBFF02E011
:10860000FFF7E8FF5B1E012803D0002B00D10520F7
:1086100000BD002BF4D1FAE770B505464FF43026C3
:108620003046FFF7E8FF042811D11C4C206940F0C8
:10863000020020616561206940F040002061304601
:10864000FFF7D9FF216941F6FD721140216170BD2C
:10865000F0B505464FF4005C0E466046FFF7CBFFD1
:10866000042814D10D4C206940F0010020612E80B7
:108670006046FFF7C0FF41F6FE77042804D1300CB6
:1086800068806046FFF7B7FF216939402161F0BD7E
:108690000249C8607047000023016745002002407E
:1086A000AB89EFCD14481549026800608A4203D0B7
:1086B0001348804713480047134E4FF009003060BD
:1086C0001248016821F07061016041020160104CA4
:1086D000182020600F49104808601048D0F800D0DA
:1086E00040680047FEE7FEE7FEE7FEE7FEE7FEE73D
:1086F000FEE7FEE7FEE7FEE7F04F0020EFBEADDE4F
:10870000ED770008ED000008181002400400014059
:10871000140C0140000C01404434434400F0FF1F9E
:10872000F0B50026012400E04C43B0FBF4F58D4287
:10873000FAD217E0B0FBF4F504FB1500B4FBF1F43A
:108740001EB9002D01DC002CF4D10A2D01DA3027EE
:1087500004E00AB1412700E061270A3F3D4403F8E5
:10876000015B761C002CE5D100201870F0BDF0B53F
:108770000026012400E04C43B0FBF4F58D42FAD210
:1087800018E000BFB0FBF4F504FB1500B4FBF1F4F6
:108790001EB9002D01DC002CF4D10A2D01DA30279E
:1087A00004E00AB1412700E061270A3F3D4403F895
:1087B000015B761C002CE5D100201870F0BD2DE97E
:1087C000F0418046069C0E4615460BB1302700E06E
:1087D0002027204600E06D1E10F8011B29B1002D56
:1087E000F9DC02E039464046B047281EA5F10105F4
:1087F000F8DC01E04046B04714F8011B0029F9D12C
:10880000BDE8F0812DE9FF5F83468A46144699460C
:108810002D2701AE83E025297ED14FF0000814F802
:10882000011B42464546302903D114F8011B4FF085
:108830000108A1F13000092818D80A23002505E015
:10884000984213DC05FB030514F8011BA1F130006D
:10885000092809D93138052801D80A3004E0A1F1E6
:108860004100052802D80A300028E9DA6C2902D133
:1088700014F8011B012264291DD008DC002953D003
:10888000252949D058292CD0632948D141E07329A2
:108890004CD0752902D0782941D122E059F8040B37
:1088A00001AB92B91AE0434600962A465146584613
:1088B000FFF785FF33E059F8040B01AB42B1002804
:1088C00003DA40428DF804705B1C00220A2110E09C
:1088D000002803DA40428DF804705B1C00220A2154
:1088E00012E059F8040B52B1582905D0002201AB0F
:1088F0001021FFF715FFD6E70122F8E70CE0582911
:1089000005D0002201AB1021FFF731FFCBE7012298
:10891000F8E759F8041BC9B258465246904714F874
:10892000011B00297FF477AFBDE8FF9F59F8041BB6
:1089300000230091B9E70A4AC2E9001070470FB45A
:10894000074810B5D0E9001003AB029AFFF75AFFB1
:10895000FEF753F90028FBD010BC5DF814FB0000B3
:10896000C8040020004870479CB70008A0F16101CE
:10897000192900D8203870472DE9F05F83460F464B
:10898000154699464FF0FF36DDF828A011E0A819EA
:10899000441009FB047080460146584652469047F1
:1089A000002802D004DA254603E04046BDE8F09FE7
:1089B0002646A5EB06000128E9DC0020F6E740EAA0
:1089C00001039B0703D009E008C9121F08C0042A4D
:1089D000FAD203E011F8013B00F8013B521EF9D234
:1089E0007047D2B201E000F8012B491EFBD270475C
:1089F0000022F6E710B50446084611460246204616
:108A0000FFF7EFFF204610BD034600E0401C027850
:108A1000002AFBD111F8012B00F8012B002AF9D113
:108A20001846704730B50EE003460A4601E05B1C6D
:108A3000521C1C781578AC4201D1002CF7D115F0EE
:108A4000FF0F04D0401C0278002AEDD1002030BD79
:108A500010B5044604E00B7800F8013B03B1491C53
:108A6000521EF8D2204610BDCAB20178914203D0FE
:108A700009B1401CF9E7002070470146002000E0E2
:108A8000401C0A5C002AFBD170472DE9F0410546E5
:108A900000200E469046044600E0641C44450BD27C
:108AA000285D00F05AFB0746305D00F056FB381A8F
:108AB00002D1295D0029F0D1BDE8F08170B50646EC
:108AC00000F0ACFD046805460A220021304600F0A3
:108AD0004AFB2C6070BDF0B480EA0102D20F430063
:108AE000B3EB410F02D20346084619464B0042D071
:108AF000C30DDDB2C1F3C7542C1B202C35DAC1F3F2
:108B0000160141F4000502B16D42C4F1200605FAD8
:108B100006F125412844B3EBD05F23D0C2B1012C2C
:108B2000A0EBC35009DCF0BC4FF0004202EAC35294
:108B300000F50000DBB200F057BB400000F1807090
:108B400000EBC350A0F1807040EAD170490009E009
:108B5000490841EAC071A0EBC35000F5000040088D
:108B600000EBC350F0BC00F036BB5142012303EBD5
:108B70004101801AF6E7F0BC704781F00041AAE796
:108B800080F00040A7E780EA010210B502F0004241
:108B9000400026D04B0023D04FEA106101EB136157
:108BA000C0F35600C3F3560340F4000043F400033F
:108BB000A0FB0330A1F17F014FEA00401C0401D06B
:108BC00000F1010050EA134001D44000491EC3B235
:108BD0000C0604EBD010401C4008802B02D003E0B0
:108BE000002010BD20F00100002900DA0020104311
:108BF00010BD80EA010202F0004330B430F00042C0
:108C000021F0004015D0A0B1C0F3C755C2F3C7543E
:108C1000C2F31601C0F31600651B41F4000140F4D5
:108C200000007D35814201D36D1C00E04900002D1C
:108C300002DA30BC002070474FF400020024814269
:108C400001D3091A144352084FEA4101F7D151B137
:108C5000814202D14FF0004105E002D24FF0010104
:108C600001E06FF0010104EBC55030BC184400F086
:108C7000B2BA420005D0C0F3C7525242914201DC61
:108C80000020704700EBC15070472DE9FE4F0746AA
:108C900081EA0300C00F0E46019021F0004123F04D
:108CA0000044B81AA14105D23846314617461E463F
:108CB0000B46024623F00040104304D138463146AB
:108CC00003B0BDE8F08F350DC5F30A00C3F30A51B8
:108CD0000290401A0090402868DAC3F3130040F471
:108CE000801B0198924620B10023D2EB030A63EB6C
:108CF0000B0B00985946C0F14002504600F0FCF9B9
:108D000080460C4650465946009A00F014FAC019A5
:108D10007141EF1785EA11533B4340D0019A52B39A
:108D2000009A012A11DC0022801A4FF0004361EB07
:108D3000055103EA05538018CDE9002341F5801160
:108D40004246234600F0D7FABAE72E050025401B1D
:108D500061EB0601401941F58012001852412818B4
:108D6000A6F5001343EB020140EAD470294318EB47
:108D70000808644113E064084FEA38084FF0000225
:108D800044EAC0744FEA0553801A61EB030180186E
:108D900041F5801149084FEA300080185941424698
:108DA000234603B0BDE8F04F00F098BA01980122C5
:108DB00040000023D0EB020263EBE07301984FEA1E
:108DC000E074381A66EB0401EBE783F000435CE7DC
:108DD00081F0004159E72DE9FE4F81EA030421F0BB
:108DE000004504F0004423F000414FF0000A0094D5
:108DF00050EA050302D052EA010304D100200146E3
:108E000003B0BDE8F08FC1F30A53C5F30A541C4404
:108E1000A0FB02B3C5F3130545F4801CC1F3130195
:108E200041F480180CFB023300FB083EA4F2F3343B
:108E3000810A930A41EA8C5143EA88530194A1FBC9
:108E400003474FEA9C2505FB03734FEA982601FB75
:108E500006373D05260545EA1435BBEB06016EEBEA
:108E60000503850E920E45EA8C1542EA8812A5FB91
:108E70000206261E67EB00070C0D44EA0334A41912
:108E800047EB1350C1F313064FF0000319464FEAA6
:108E9000033343EA165343EA0403019CE5FB020152
:108EA000A4F10C040294009C4FEA0632CDE900A420
:108EB00000F021FAA4E72DE9F04D81EA030404F063
:108EC000004B21F0004714464FF0000A23F0004108
:108ED00050EA070220D054EA01021DD0C1F30A551E
:108EE0000246C1F31300C7F30A56C7F3130340F455
:108EF000801143F48013A6EB0508101BD64608F238
:108F0000FD3873EB010002D308F1010801E092186B
:108F10005B41B8F1000F03DA00200146BDE8F08D97
:108F200000204FF48015064607460EE0B2EB040C15
:108F300073EB010C04D3121B064363EB01032F43B5
:108F40006D084FEA300092185B4150EA050CEDD1F4
:108F500052EA030012D082EA040083EA01052843A2
:108F600003D100224FF0004308E0101B8B4102D2D6
:108F70000122002302E06FF0010253101AEB0600F9
:108F800047EB085110EB0A0041EB0B01BDE8F04D37
:108F900000F0A4B9C10F80EAE0700844CA07962324
:108FA000002100F021B996230022114600F01CB9DF
:108FB0000EB5C10F80EAE0700844CA07002140F2F4
:108FC00033438DE80E000A460B4600F094F903B0D7
:108FD00000BD00F0004220F00040C10DC0F31600BB
:108FE00040F400007F2901DA00207047962903DC55
:108FF000C1F19601C84001E096398840002AF4D0BA
:109000004042704720F00040C10DC0F3160040F40C
:1090100000007F2901DA00207047962903DCC1F1A6
:109020009601C840704796398840704770B5C1F3C3
:109030000A5201F000450024C1F3130140F2FF334E
:1090400041F480119A4201DA002070BD40F23343AE
:109050009A42A2F2334203DC524200F05CF800E094
:1090600090402C43F1D0404270BD00F0004230F0FF
:1090700000400DD0C10D01F5607142EA015100229E
:10908000C0F31600520742EAD0024007114370476E
:1090900000200146704701F0004230B421F0004149
:1090A00050EA010306D00B0DA3F56073C1F3130161
:1090B000002B02DC30BC00207047440F44EAC1049E
:1090C000C100A01830BC00EBC35000F084B8000011
:1090D000002801DBC0F10040002901DBC1F10041A3
:1090E00081427047002801DBC0F10040002901DB0C
:1090F000C1F1004188427047202A04DB203A00FA7F
:1091000002F1002070479140C2F1200320FA03F3DE
:10911000194390407047202A04DB203A21FA02F0DC
:109120000021704721FA02F3D040C2F120029140A1
:10913000084319467047202A06DBCB17203A41FA2C
:1091400002F043EAE071704741FA02F3D040C2F105
:1091500020029140084319467047A0F141011929A6
:1091600000D8203070472DE9F0470F4691468046E1
:109170000446002614F8015B2DB1FFF7F3FB0068ED
:10918000405DC007F6D12B2D02D02D2D18D0641EC6
:109190004A463946204600F03DF927B13968A142D8
:1091A00001D1C7F8008071054FF002040BD5404291
:1091B000002803DD00F032FA0460A007BDE8F08764
:1091C00046F48066E4E70028F8DA00F027FA046045
:1091D0006FF00040F2E70029A8BF7047401C49002B
:1091E00008BF20F00100704710B4B0FA80FC00FA0C
:1091F0000CF050EA010404BF10BC704749B1CCF137
:10920000200421FA04F411FA0CF118BF01212143C2
:109210000843A3EB0C01CB1D0106000A002BBEBFC7
:10922000002010BC704700EBC35010440029A4BFBD
:1092300010BC7047401C490008BF20F0010010BC62
:109240007047F0B4002802DCF0BC00207047C0F387
:10925000C751C0F3160040F40000CA0701D1400016
:10926000491E3F2202EB6105002211464FF4000621
:1092700026FA01F31344D418844201D8001B1A467D
:109280004000491C1729F3DD5100814202D24FF002
:10929000FF3100E0002102EBC550F0BCFFF79BBF9F
:1092A00010B541000CD0C0F3C751962908DC7E29C7
:1092B00009DC06DB410204D000F0004040F07E50A3
:1092C00010BD002010BDC1F19604C4F1200100FAC8
:1092D00001F1E040FFF77FFFA04010BD10B5002B6B
:1092E00008DA401C41F1000192185B411A4301D198
:1092F00020F0010010BD2DE9F04D92469B4611B1C2
:10930000B1FA81F202E0B0FA80F220329046FFF723
:10931000F3FE06460F4640EA0A0041EA0B015246B8
:109320005B46084303D130463946BDE8F08D194607
:1093300052EA010015D0C8F140025046FFF7EBFE9B
:1093400004460D46504659464246FFF7D5FE0843AF
:1093500001D0012000E00020044345EAE0752643E7
:109360002F430A984FEAD625A0EB08000A304FEAAF
:1093700046534FF0000245EA47554FEAD72402D53D
:1093800000200146D1E7010550196141DDE908459A
:1093900000196941BDE8F04DA0E770B521F0004328
:1093A00003430CD0C1F30A540026D4EB060566EB48
:1093B0000603D417AD1AA34102DB0020014670BD9D
:1093C000001C41EB025170BD30B5002904DB4FF0A9
:1093D0000044404264EB0101002B04DB4FF00044E9
:1093E000524264EB0303994208BF904230BD000033
:1093F000064C074D06E0E06840F0010394E80700E2
:1094000098471034AC42F6D3F6F774FEDCBE000881
:10941000FCBE00082DE9F05F8246007800278B46ED
:1094200015460AF10104B946302801D09DB113E078
:1094300014F8010B0127782803D0582801D045B132
:109440000AE00DB1102D07D10027102514F8010BEB
:1094500002E0082500E00A250026B0460EE005FBE4
:10946000080005FB06F1012701EB10461FFA80F802
:10947000B6F5803F00D3B94614F8010B294600F039
:1094800069F80028EBDABBF1000F05D00FB1641EBC
:1094900000E05446CBF80040B9F1000F06D000F0D0
:1094A000BDF802210160C81EBDE8F09F48EA0640F1
:1094B000FAE72DE9F04D00231A461B1A8A4103DB17
:1094C00000200146BDE8F08DC1F30A52C1F313013B
:1094D00041F480154FF0000BD10702D100186D4107
:1094E000521E0026044640F2FF11304601EB620A8C
:1094F00037468046024600204FF48011FFF70BFEEE
:1095000080197941331847EB0102B4EB030C75EB7A
:10951000020C04D3E41A65EB020506460F46241933
:1095200008F101006D4180463428E3DDB11947EBB5
:109530000700091BA84103D24FF0FF32134601E098
:10954000002213461BEB060047EB0A51BDE8F04D25
:10955000FFF7C4BE3A2800D2303820F02002412A5A
:1095600001D3A2F13700884201D34FF0FF3070479A
:1095700070B501EB020410F8015B15F0070301D18F
:1095800010F8013B2A1106D110F8012B03E010F866
:10959000016B01F8016B5B1EF9D12B0705D4002389
:1095A000521E0FD401F8013BFAE710F8013B02F11B
:1095B0000202A1EB030303E013F8015B01F8015B76
:1095C000521EF9D5A142D6D3002070BD490050EA01
:1095D000C12018BF04204A0D18BF40F0010040F21E
:1095E000FF72B2EB515F08BF40F00200012808BFD4
:1095F000052070474100080218BF04200A0E18BF5A
:1096000040F001004FF07F4232EA010108BF40F014
:109610000200012808BF052070470000004870477D
:10962000D00400202DE9F0414F1E00EBC701044695
:10963000D1E9000115461E4637F006020DD02A4634
:109640003346FFF7C8FB7F1E04EBC703D3E90023B3
:10965000FFF71BFB37F00602F1D1022F25D0042FB4
:1096600013D0062F18BFBDE8F0812A463346FFF716
:10967000B2FBD4E90A23FFF708FB2A463346FFF77B
:10968000AAFBD4E90823FFF700FB2A463346FFF77D
:10969000A2FBD4E90623FFF7F8FA2A463346FFF780
:1096A0009AFBD4E90423FFF7F0FA2A463346FFF782
:1096B00092FBD4E90223FFF7E8FA2A463346FFF784
:1096C0008AFBD4E90023BDE8F041FFF7DEBA0000D1
:1096D000024A00201107FFF760BE000001FDFFFFF6
:1096E0006FF05E010807FFF7C4BA00002DE9F04DE6
:1096F000034614464FF07F400E46B0EB440F04D8AB
:10970000001608601846BDE8F08D4FF0004040EAB2
:109710000421C4F3C7507838431100F01F00DFF86C
:1097200014C1C0F12002FC445CF823500CEB83030D
:109730008540D3F804C02CFA02F72F439D680CFA39
:1097400000FC25FA02F8DB6805FA00F023FA02F2C1
:1097500040EA02054CEA080CA7FB0123ACFB01C060
:10976000A5FB015101EB0C05A94294BF4FF0000C81
:109770004FF0010C81186144BCF1000F02D081420E
:1097800002D903E0814201D2012000E00020184408
:1097900000F120024FEA92188006CA0C40EA4230DB
:1097A0004F03C6F80080FFF7F5FB82463846FFF707
:1097B000FAFB6FF01201FFF75CFA07462846FFF745
:1097C000F2FB6FF02501FFF754FA83463946504605
:1097D000FFF781F95946FFF77EF900F500656FF351
:1097E0000B0551462846FFF7C8F93946FFF7C5F97A
:1097F0005946FFF7C5F91049FFF7C5F907460F4964
:109800002846FFF7C0F93946FFF765F907460C49C6
:109810002846FFF7B8F93946FFF75DF914F0004F15
:1098200008BFBDE8F08DC8F1805180F00040316084
:10983000BDE8F08D7E200000DB0FC92F22AAFD2994
:109840000000C92F02E008C8121F08C1002AFAD17F
:1098500070477047002001E001C1121F002AFBD1B0
:10986000704700000149086070470000D0040020E4
:109870002DE9F04104464FF00E4000EB4400B0F1FA
:10988000506F204620D94FF0E441B1EB440F08D986
:10989000FFF7B0FE042808BFFFF722FF2046BDE80F
:1098A000F0814FF07F41B1EB440F04D2BDE8F041AD
:1098B0000121FFF7DEB90120FFF7D4FFBDE8F04139
:1098C00000210846FFF795B94FF0FC41B1EB440F7A
:1098D0001CD224F000404FF07E51FFF751F94FF0B9
:1098E000FF31FFF7C6F9054601F022F814F0004FEA
:1098F0001DBF204E204F80F00040204E08BF204F5B
:109900004FF04041FFF73FF9044605E00026374697
:109910000146FFF738F905461A492846FFF733F99B
:109920001949FFF7D8F82946FFF72DF91749FFF72E
:10993000D2F82946FFF727F91549FFF7CCF8294651
:10994000FFF721F91349FFF7C6F88046294620465C
:10995000FFF719F94146FFF716F905463946204643
:10996000FFF7B9F82946FFF7B6F83146BDE8F041F0
:10997000FFF7B1B80000C9BF22AAFDB90000C93F76
:1099800022AAFD3924FE1C3DC78AD83C1E67383DFB
:109990001B93993DAFAA2A3E2DE9F0474FF068424C
:1099A00002EB400305460C46B3F1654F3CBF02EBAA
:1099B0004102B2F1654F3FD34FF07F42B2EB400F0F
:1099C00028BFB2EB410F03D2BDE8F047FFF783B8E1
:1099D00040EA01035B0008BF44F0FF410AD0B2EB4C
:1099E000400F08BFB2EB410F06D125F0804024F0B4
:1099F000804105460C461FE0B2EB400F12BF5FEA04
:109A0000410245F0FF4004F0004115D04FEA410209
:109A100092EA400310D4002AACBF4FF09F464FF0AB
:109A20003E563146FFF7AFF8054631462046FFF770
:109A3000AAF8044628462146C0F3C752C1F3C753CB
:109A4000D21A1B2A06DD10F0004F14BF54485548A7
:109A5000BDE8F08712F11A0F17DA11F0004F06D0A7
:109A600010F0004F14BF50485048BDE8F087214621
:109A70002846FFF7BEF80446FFF7BCFD042808BFE0
:109A8000FFF72EFE2046BDE8F0874200B2EB410F03
:109A900025D910F0004F19BF454F464E464F474E4F
:109AA000224685F0004415460A4680F000411046E3
:109AB0000A1A5200B2F1807F3ED248404049DFF896
:109AC00004A110F0004F18D04FF03F483846FFF780
:109AD00054F8074651463046FFF74FF817E011F0AB
:109AE000004F04BF00263746E2D010F0004F19BFE8
:109AF000354F364E364F374EDAE74FF07C58384602
:109B0000FEF7E9FF074651463046FEF7E4FF0646FA
:109B100041462846FFF737F82146FEF7DCFF82462C
:109B200021464046FFF72FF82946FFF729F851460E
:109B3000FFF75FF8044604E021462846FFF759F88E
:109B400004460146FFF71FF880462349FFF71BF83C
:109B50002249FEF7C0FF4146FFF715F82049FEF7FE
:109B6000BAFF4146FFF70FF81E49FEF7B4FF414622
:109B7000FFF709F81C49FEF7AEFF054641462046AF
:109B8000FFF701F82946FEF7FEFF3146FEF7A3FF77
:109B90002146FEF7A0FF3946BDE8F047FEF79BBF20
:109BA000DB0FC9BFDB0FC93FDB0F49C0DB0F4940EB
:109BB0000000C9BF22AAFDB90000C93F22AAFD3991
:109BC0000060ED3EC30ACE37000049C022AA7DBA2C
:109BD0000000494022AA7D3A2DAD65BD8FB8D53D24
:109BE0000FB511BE61C84C3EA8AAAABE2DE9F84324
:109BF0000446024650486946B0EB420F09D94FF07F
:109C0000E640B0EB420F8CBF4FF0FF3000200090D9
:109C100034E04A4B22F0004083422BD94849204689
:109C2000FEF7B1FFFFF73CFB0546FFF7D2F900F066
:109C30000300009043492846FEF7A5FF0646424927
:109C40002846FEF7A0FF074640492846FEF79BFF3F
:109C500080463F492846FEF796FF2146FEF790FFD3
:109C60004146FEF78AFF3946FEF787FF3146FEF789
:109C700084FF02E01046FFF739FD0446009D002DE9
:109C800018DA6000B0F17F4F3CBF4FF07E50BDE866
:109C9000F88309D14FF00100FFF7E4FDBDE8F84378
:109CA00000210846FEF7A5BF2046BDE8F843012184
:109CB000FEF7DFBF214615F0010F08461DD0FEF765
:109CC00062FF06462349FEF75EFF2349FEF758FF71
:109CD0003146FEF758FF2149FEF7FDFE3146FEF7FB
:109CE00052FF2146FEF74FFF2146FEF7F4FE15F026
:109CF000020F18BFBDE8F8831AE0FEF744FF0446E0
:109D00001749FEF740FF1749FEF7E5FE2146FEF72B
:109D10003AFF1549FEF7DFFE2146FEF734FF4FF00C
:109D20007E51FEF7D8FE15F0020F08BFBDE8F8839C
:109D300080F00040BDE8F883B61F927E490E494688
:109D400083F9223F1A61342C0020A23300A0FD3990
:109D50000000C93F336D4C39DA82083CA0AA2ABE04
:109D6000B93AB2BACA9F2A3DDDFFFFBE2DE9F04DD8
:109D700016460F460546020096B01C4621F00041EB
:109D800023F0004014BF4FF0010C4FF0000C0CEB1F
:109D9000470CFE4B0CEB03084FEA630CC4452DD86F
:109DA0005FEA060818BF4FF0010808EB4408984422
:109DB000F74B434522D8F74B50EA060C02D09F429E
:109DC00005D14AB916B000201946BDE8F08D002A29
:109DD00008BF4FF0000C01D04FF0010C0CEB470313
:109DE00013F5001F0AD8002E14BF4FF0010C4FF0DE
:109DF000000C0CEB440313F5001F08D916B03246D3
:109E0000234628463946BDE8F04DFEF73EBFDFF851
:109E100088B34FF0000A002FB8BF584523DADF4B54
:109E20009842A8BF4FF0020A1DDADA4B98421ADBBB
:109E3000DB4B03EB2053142B08DDC3F1340C26FA63
:109E40000CF303FA0CFCB4450DD108E05EB9C3F184
:109E5000140C20FA0CF303FA0CFC844503D103F034
:109E60000103C3F1020A51EA020321D1002C1FDAD7
:109E7000002F18BFBAF1020F02D0BAF1010F0BD0B8
:109E80000220FFF7EFFC16B00022BDE8F04D1346AC
:109E90001046C049FFF70FB80220FFF7E3FC16B0E9
:109EA0002A463B46BDE8F04D0020BA49FFF703B80B
:109EB000330076D1584525D107F1804010F5801048
:109EC00001BF002A0020B34916B008BFBDE8F08DDD
:109ED000B048814207DB002CA1BF1846214616B0CE
:109EE000BDE8F08D07E0201E05DA80F0004116B0D5
:109EF0001846BDE8F08DAB497944D1E9000116B0B0
:109F0000BDE8F08DDFF88CC260452FD1002C28DA37
:109F100039B159451CD1002A04BF002002460CD09B
:109F20001FE06AB10220FFF79DFC40F201320020E1
:109F30004FF0E041FFF731FA0A46394600F0DEBA49
:109F4000954A394616B0002062F31E01BDE8F08D37
:109F500007DA16B03B46BDE8F04D00206146FEF73B
:109F6000AABF16B010463946BDE8F08D8B4518DD06
:109F7000B4F1804F0DD0A4F10053B3F1FF5310D1D1
:109F80003B1E0EDB16B01046BDE8F04D194600F042
:109F9000A9BC3B4616B01046BDE8F04D1946FEF789
:109FA0001ABF27F00043A2BBE1B1594538D1002FB9
:109FB00006DD002CA1BF0020594616B0BDE8F08D8B
:109FC000002F01DD002C1FDB002F16DA002C14DB24
:109FD000BAF1010F4FF000000CBF73496E4916B083
:109FE000BDE8F08DBAF1020F18BF002F0CD0BAF106
:109FF000010F09D1002F07DA0CE0002FB8BF002CA9
:10A000000EDABAF1010F05D0002016B00146BDE806
:10A01000F08D05E016B000204FF00041BDE8F08D56
:10A020004FF0010C0CEBE7720F9252EA0A020BD0D0
:10A030005E4A90427DDD5E4B5E4A984216DD91425B
:10A040000EDC002C1CDB2CE00120FFF70BFC16B013
:10A050000022BDE8F04D134610461146FEF72BBF17
:10A060004C48884202DC002C0ADC1AE08A4202DDFD
:10A07000002C05DB15E0474B99421EDD002C10DD5E
:10A080000220FFF7EFFB40F2013200204FF0E041E9
:10A09000FFF783F9404A16B061F31E021146BDE88E
:10A0A000F08D0220FFF7DEFBFFF712FB394A16B0F6
:10A0B00061F31E021146BDE8F08D002228463946A4
:10A0C000FEF783FE05460F466FF00102FFF765F9C4
:10A0D0004FF05532384BFEF77BFE2A463B46FEF7E3
:10A0E0007AFE0022354BFEF773FE8B4680462A46E9
:10A0F0003B4610461946FEF76EFE42465B46FEF7AB
:10A100006AFE80460B914FF0C0422D4B28463946DF
:10A11000FEF761FE834605912A4A294B40460B997A
:10A12000FEF759FE88460290274A284B28463946B2
:10A1300000E01BE0FEF74FFE4346029AFEF745FEA5
:10A14000054602460B460B9158460599FEF79DFDC4
:10A15000002788465A463846059BFEF736FE2A46B3
:10A160000B9BFEF735FE024600F073B90020B1F5F7
:10A17000801F07DA352228461946FFF70EF90546F3
:10A180006FF0340000EB215022E00000FFFF1F00C1
:10A19000FFFF0F000000F03F0000F07F0000404391
:10A1A00001FCFFFFA41800000000F0FF0000E041E8
:10A1B0000000F043FFFFEF3F5555D53F0000E03F63
:10A1C0004715F73FFE822B6544DF5DF80BAE543E2A
:10A1D000A0F2FF300190C1F3130040F07F6141F025
:10A1E00040510291FE498842D8BF4FF0000B0EDD6E
:10A1F000FC498142C8BF4FF0010B08DC01984FF0C9
:10A20000000B401C01900298A0F580100290F648C7
:10A210000299784400EBCB0009910790D0E9002324
:10A220002846FEF7D2FD059100900798D0E900235B
:10A2300028460999FEF729FD02460B460020EB4906
:10A24000FEF739FE0B910B460246069005990098E1
:10A25000FEF7C1FD0A90E64888460027784400686A
:10A260000C9002994FF0005040EA610000EB8B40E7
:10A2700000F5002102910798D0E900230C98FEF721
:10A28000A4FD2A46099BFEF7A3FD3A464346FEF786
:10A29000A2FD0791054638464146029B0C9AFEF7FF
:10A2A0009AFD059B009AFEF793FD2A46079BFEF751
:10A2B0008CFD0B9B069AFEF78EFD0A9A069108907C
:10A2C000434610461946FEF786FD05460246C94834
:10A2D0000B46079106217844FFF7A4F90290079BEB
:10A2E0002A46059110461946FEF775FD059B029A10
:10A2F000FEF771FD059105464346384619460A9A10
:10A30000FEF7C3FC069B089AFEF765FD2A46059BEF
:10A31000FEF7BBFC3A46434605911290104619469B
:10A32000FEF759FD0022B44B07910090FEF7ADFCFB
:10A33000059B129AFEF7A9FC0D463A46AE4B3846ED
:10A34000FEF743FD079B009AFEF73FFD059B129A1F
:10A35000FEF73EFD3A46079112902B4610464146C5
:10A36000FEF739FD0591009043460A9A0799129825
:10A37000FEF731FD804607912B463A46069908982C
:10A38000FEF729FD4246079BFEF77FFC88460690B4
:10A39000059B009AFEF779FC00200F460546059BB9
:10A3A000009AFEF712FD4346069AFEF711FD80461D
:10A3B0000D914FF06042914B28463946FEF70BFD58
:10A3C000059100908E4A8D4B40460D99FEF703FD96
:10A3D000804604918B4A8C4B28463946FEF7FBFC9D
:10A3E0004246049BFEF751FC884A7A4402EBCB03B9
:10A3F000D3E90023FEF749FC029004910198FEF78F
:10A40000D7FD0791DDE904310546029A0098FEF771
:10A410003CFC7F4A7A4402EBCB0BDBE90023FEF7DE
:10A4200034FC2A46079BFEF730FC002788462A4664
:10A430003846079BFEF7C9FCDBE90023FEF7C5FCA5
:10A44000059B009AFEF7C1FC049B029AFEF7C0FC34
:10A45000024600200A900F98644DAAF101031843A8
:10A4600001D16C4D0A9000200B46029030462146E7
:10A47000FEF7B1FC82468B46234630461946029AC7
:10A48000FEF7A3FC3A464346FEF7A5FC52465B4660
:10A49000FEF7FBFB06468A463A46434621460298AB
:10A4A000FEF799FC04460F4632465346FEF7EDFB95
:10A4B000594A8B46914226DBABEB020353EA00027A
:10A4C00010D122463B46FEF780FC80460391534A5A
:10A4D000534B30465146FEF7D8FB4246039BFEF7EE
:10A4E00073FF2CD20220FFF7BDF940F201320020A9
:10A4F0004FF0E041FEF751FF0A46294616B062F3DD
:10A500001E01BDE8F08D474B2BF000429A4216D356
:10A51000454A0BEB020353EA000208D122463B46B0
:10A52000FEF753FC32465346FEF74EFF07D8022093
:10A53000FFF798F9FFF7CCF80A462946DEE72BF03B
:10A5400000403A493A4A01EB20514FF0000890424E
:10A5500023DD481C4FF4801121FA00F05844C0F369
:10A560000A51344AA1F2FF317A44334B1268CB408E
:10A5700020EA0303C0F3130040F4801CC1F114006F
:10A580002CFA00F8BBF1000FB8BFC8F10008204654
:10A590003946FEF71AFC04460F4622463B46304633
:10A5A0005146FEF772FB4FF0000B5A46234B5846BC
:10A5B0000791FEF710FC05910090214A214B584667
:10A5C0000799FEF708FCCDE9020122463B465846B2
:10A5D0000799FEF7FAFB32465346FEF7F9FB33E0E4
:10A5E0008E9803007AB60B007A1400000000F03F4A
:10A5F00040150000E61300000000084009C7EE3FC8
:10A60000FD033ADCF5015B14E02F3EBEC2120000F0
:10A61000881200000000F0BF00009040FE822B6511
:10A620004715973C00CC904000346F3F01FCFFFF82
:10A630000000E03F34120000FFFF0F00432EE63F12
:10A64000396CA80C615C20BE3F4A404BFEF7C3FB4F
:10A65000DDE90223FEF719FB07468A46059B009AAF
:10A66000FEF713FB04460E46059B009AFEF7ADFB72
:10A670003A465346FEF7ACFB0746224633460B915B
:10A6800010461946FEF7A7FB8346024630488A4625
:10A690000B4605217844FEF7C5FF5A465346FEF7A0
:10A6A0009AFB22463346FEF793FB82468B463A4698
:10A6B000204631460B9BFEF78EFB3A460B9BFEF77E
:10A6C000E4FA00910C9000224FF080435046594626
:10A6D000FEF77BFB0746039152465B462046314618
:10A6E000FEF779FB3A46039BFEF7E5FB009B0C9ACD
:10A6F000FEF76BFB22463346FEF767FB0022154B45
:10A70000FEF766FB0E46044601EB085108150028CB
:10A7100010DC424620463146FEF73FFEFEF756FF6C
:10A72000042808BFFEF7D4FF424620463146FEF714
:10A7300034FE04460A980B4616B022462946BDE868
:10A74000F04DFEF748BB0000EF39FAFE422EE63F1F
:10A75000581000000000F03F2DE9F843044654482B
:10A7600022466946B0EB420F09D94FF0E640B0EB04
:10A77000440F8CBF4FF0FF300020009034E04D4B71
:10A7800022F0004083422BD94B491046FEF7FBF9DB
:10A79000FEF786FD0646FEF71CFC00F00300009065
:10A7A00046493046FEF7EFF9054645493046FEF783
:10A7B000EAF9074643493046FEF7E5F98046424943
:10A7C0003046FEF7E0F92146FEF7DAF94146FEF79A
:10A7D000D4F93946FEF7D1F92946FEF7CEF902E061
:10A7E0001046FEF783FF0446009D002D1DDA600031
:10A7F000B0F17F4F09D22046FEF7FCFE042808BFC7
:10A80000FEF76EFF2046BDE8F88308D10120FFF770
:10A8100029F8BDE8F84300210846FEF7EAB92046CA
:10A82000BDE8F8430121FEF724BA214615F0010FD7
:10A8300008461FD0FEF7A7F904462449FEF7A3F9FE
:10A840002349FEF748F92146FEF79DF92149FEF715
:10A8500042F92146FEF797F94FF07E51FEF73BF99A
:10A8600015F0020F08BFBDE8F88300BF80F000407C
:10A87000BDE8F883FEF787F906461749FEF783F926
:10A880001649FEF77DF93146FEF77DF91449FEF7CA
:10A8900022F93146FEF777F92146FEF774F9214691
:10A8A000FEF719F915F0020FE0D1BDE8F8830000BA
:10A8B000B61F927E490E494683F9223F1A61342C15
:10A8C0000020A23300A0FD390000C93FB93AB2BA56
:10A8D000CA9F2A3DDDFFFFBE336D4C39DA82083C4A
:10A8E000A0AA2ABE2DE9F04106460F46FEF7E1FD7B
:10A8F0000D46040018BF0120284320F00040C0F19D
:10A900007F6010F1E0400FD5002E14BF0120002021
:10A91000384320F00040C0F17F6000F1E0400028A3
:10A92000A4BF0120FEF79EFF20462946BDE8F08126
:10A9300070B50546FEF785FC044620F00040C0F1E6
:10A94000FF40C00F08D025F00040C0F1FF40C00F0D
:10A9500004BF0120FEF786FF204670BDC4BD00087D
:10A960005BBC000875030008ABBC000800BD000814
:10A970004D060008D9BC0008FFBD00089506000878
:10A98000E6B9000805BB0008BB06000817BC0008B4
:10A99000FFBD00088707000813BC00083FBC000883
:10A9A000B107000869BC00081DBD000825080008A3
:10A9B00037BA0008F0BC000871060008D5BC0008D2
:10A9C00030BD000835090008CEBC0008C2BC000834
:10A9D000610C0008CEBB0008FFBD0008EF0C0008AA
:10A9E0003CB90008000000008D05002000000000B8
:10A9F0002000000039B90008000000008E0500208A
:10AA00000000000064000000EBBA00080000000035
:10AA10008F05002001000000FA000000D6B80008F1
:10AA20000200000092050020B0040000A40600000F
:10AA3000AFB90008020000009E05002000000000E1
:10AA4000D0070000BBB9000802000000A0050020EC
:10AA500000000000D007000045B900080200000017
:10AA6000A205002000000000D0070000B6BA0008D0
:10AA7000020000009405002000000000D007000044
:10AA8000BFBA000802000000960500200000000088
:10AA9000D007000046BB0008000000009805002019
:10AAA0000000000001000000C9BD00080000000017
:10AAB0009905002000000000C8000000D8BD000873
:10AAC000000000009A05002000000000C8000000FF
:10AAD0009DB90008020000009C050020E80300006A
:10AAE000D0070000FDB9000802000000A405002006
:10AAF00032000000F2010000EEB900080200000080
:10AB0000A605002032000000F20100001ABA000879
:10AB100004000000FC050020B004000000C2010099
:10AB20002ABA000804000000EC050020B004000070
:10AB300000C201008FBC000800000000900500204A
:10AB4000000000000100000084B9000800000000BF
:10AB5000820500200A000000C800000063B9000858
:10AB600000000000830500200A0000003200000001
:10AB700050B9000800000000840500200A00000011
:10AB800032000000E6BB000801000000C005002004
:10AB9000FFFFFFFF010000008EB900080200000067
:10ABA000C205002000000000D0070000C2BB000862
:10ABB00002000000C405002000000000D0070000D3
:10ABC000B8BD000802000000C6050020000000001B
:10ABD000D0070000A5BB000802000000C805002047
:10ABE00000000000D00700001CB9000802000000AF
:10ABF000CA05002000000000D00700009BBD00082F
:10AC000002000000CC05002000000000D00700007A
:10AC1000B3BB000802000000CE05002000000000C9
:10AC2000D00700002AB9000802000000D00500206B
:10AC300000000000D0070000A9BD000802000000CD
:10AC4000D205002000000000D0070000C8BA0008AC
:10AC500001000000D4050020FFFFFFFF01000000FD
:10AC60001CBC000801000000D5050020FFFFFFFF0D
:10AC700001000000DABA000801000000D60500203B
:10AC8000FFFFFFFF010000002EBC000801000000D4
:10AC9000D7050020FFFFFFFF010000009EBC000859
:10ACA00000000000DA05002000000000FF000000A6
:10ACB00053BB000801000000D80500209CFFFFFFE7
:10ACC0006400000065BB000801000000D9050020F9
:10ACD0009CFFFFFF6400000084BB0008020000002E
:10ACE000DC05002064000000B80B00007ABD0008FD
:10ACF00002000000DE05002064000000B80B000028
:10AD0000FBB8000802000000E0050020640000001D
:10AD1000B80B000095BB000802000000E20500200F
:10AD200064000000B80B00008BBD000802000000AA
:10AD3000E405002064000000B80B00000CB9000816
:10AD400002000000E605002064000000B80B0000CF
:10AD5000D9B90008000000004A05002000000000EA
:10AD6000030000006FBC0008000000004B0500203D
:10AD700000000000FA000000EBBD00080000000029
:10AD80004C05002001000000FA00000061BA000834
:10AD9000020000004E05002000000000000100003D
:10ADA0007EBC000802000000500500206400000086
:10ADB000E803000076B900080000000058050020F4
:10ADC00000000000010000003CBA00080000000084
:10ADD00059050020000000003000000052BA0008B1
:10ADE000050000005C0500200000000001000000DC
:10ADF0004ABA0008050000006005002000000000BD
:10AE000001000000D6BB000803000000440500203C
:10AE1000B0B9FFFF50460000D0B9000800000000A4
:10AE2000E80500200000000003000000FFBB000850
:10AE3000000000001605002000000000C80000000F
:10AE4000A2BA000800000000200500200000000059
:10AE5000C8000000E7B80008000000002A05002034
:10AE600000000000C8000000F4BB00080000000063
:10AE70001705002000000000C800000097BA000875
:10AE8000000000002105002000000000C8000000B4
:10AE9000DCB80008000000002B05002000000000C6
:10AEA000C800000009BC00080000000018050020D0
:10AEB00000000000C8000000ACBA0008000000005C
:10AEC0002205002000000000C8000000F1B80008C2
:10AED000000000002C05002000000000C800000059
:10AEE000B4BC000802000000F005002000000000D3
:10AEF000D00700006ABA000800000000F405002036
:10AF0000000000000100000076BB00080200000005
:10AF1000F60500200A000000D00700006CBD000804
:10AF200002000000F80500200A000000D007000021
:10AF30000CBA000800000000F3050020000000002B
:10AF400064000000C7B900080200000010050020DE
:10AF500000000000282300008FBA00080000000055
:10AF60001305002000000000C800000087BA000898
:10AF7000000000001D05002000000000C8000000C7
:10AF80007FBA000800000000270500200000000034
:10AF9000C80000003FBB00080000000012050020B0
:10AFA00000000000C800000038BB000800000000DE
:10AFB0001C05002000000000C800000031BB000894
:10AFC000000000002605002000000000C80000006E
:10AFD0005EBD000800000000140500200000000015
:10AFE000C800000058BD0008000000001E05002039
:10AFF00000000000C800000052BD00080000000072
:10B000002805002000000000C8000000EABC00087D
:10B01000000000001505002000000000C80000002E
:10B02000E4BC0008000000001F0500200000000034
:10B03000C8000000DEBC0008000000002905002058
:10B0400000000000C800000029BB0008000000004C
:10B050001905002000000000C800000021BB000806
:10B06000000000002305002000000000C8000000D0
:10B0700019BB0008000000002D05002000000000A2
:10B08000C800000041455254313233340000000002
:10B090000000803F00000000A8AAAA3F00000000B6
:10B0A0000000803F000080BFB0AA2ABF000000005F
:10B0B0000000803F0000803FB0AA2ABF00000000CF
:10B0C0000000803F000000000000803F000080BFC3
:10B0D0000000803F000080BF000000000000803FB3
:10B0E0000000803F0000803F000000000000803F23
:10B0F0000000803F00000000000080BF000080BF13
:10B100000000803F000080BF0000803F000080BF43
:10B110000000803F000080BF000080BF0000803F33
:10B120000000803F0000803F0000803F0000803F23
:10B130000000803F0000803F000080BF000080BF13
:10B140000000803F0000803F000000000000000081
:10B150000000803F000080BF0000000000000000F1
:10B160000000803F00000000A8AAAA3F0000803F26
:10B170000000803F000080BFB0AA2ABF000080BF4F
:10B180000000803F0000803FB0AA2ABF000080BFBF
:10B190000000803F00000000A8AAAA3F000080BF76
:10B1A0000000803F000080BFB0AA2ABF0000803F9F
:10B1B0000000803F0000803FB0AA2ABF0000803F0F
:10B1C0000000803F000080BFD0B35D3F0000803FA3
:10B1D0000000803F000080BFD0B35DBF000080BF93
:10B1E0000000803F0000803FD0B35D3F0000803F03
:10B1F0000000803F0000803FD0B35DBF000080BFF3
:10B200000000803F00000000D0B35DBF0000803F21
:10B210000000803F00000000D0B35D3F000080BF11
:10B220000000803F000000000000803F000080BF61
:10B230000000803F000080BF000080BF00000000D1
:10B240000000803F000000000000803F0000803FC1
:10B250000000803F0000803F000080BF0000000031
:10B260000000803FD0B35DBF0000803F0000803F02
:10B270000000803FD0B35DBF000080BF0000803F72
:10B280000000803FD0B35D3F0000803F000080BFE2
:10B290000000803FD0B35D3F000080BF000080BF52
:10B2A0000000803FD0B35DBF00000000000080BF01
:10B2B0000000803FD0B35D3F000000000000803FF1
:10B2C0000000803F000080BF0000803F000080BF82
:10B2D0000000803F000080BF000080BF0000803F72
:10B2E0000000803F0000803F0000803F0000803F62
:10B2F0000000803F0000803F000080BF000080BF52
:10B300000000803F000080BF0000803F0000803FC1
:10B310000000803F000080BF000080BF000080BFB1
:10B320000000803F0000803F0000803F000080BFA1
:10B330000000803F0000803F000080BF0000803F91
:10B340000000803FF704353FF70435BF0000803F21
:10B350000000803FF70435BFF70435BF0000803F91
:10B360000000803FF70435BFF704353F0000803F01
:10B370000000803FF704353FF704353F0000803F71
:10B380000000803F00000000000080BF000080BF80
:10B390000000803F000080BF00000000000080BF70
:10B3A0000000803F000000000000803F000080BFE0
:10B3B0000000803F0000803F00000000000080BFD0
:10B3C0000000803F0000803F000000BF0000803F81
:10B3D0000000803F000000BF000080BF0000803FF1
:10B3E0000000803F000080BF0000003F0000803F61
:10B3F0000000803F0000003F0000803F0000803FD1
:10B400000000803F0000003F000080BF000080BFC0
:10B410000000803F000080BF000000BF000080BF30
:10B420000000803F000000BF0000803F000080BFA0
:10B430000000803F0000803F0000003F000080BF10
:10B440000000803F000000000000803F0000803FBF
:10B450000000803F000080BF000080BF00000000AF
:10B460000000803F000000000000803F000080BF1F
:10B470000000803F0000803F000080BF000000808F
:10B4800000000000000000000301000090B0000870
:10B4900004000000C0B000080400000000B1000873
:10B4A0000201000040B1000800010000000000009F
:10B4B0000600000060B1000806000000C0B10008EE
:10B4C00001010000000000000400000020B200089C
:10B4D0000600000060B2000808000000C0B20008CA
:10B4E0000800000040B3000808000000C0B30008D6
:10B4F0000101000000000000000100000000000049
:10B5000000010000000000000400000040B400083A
:10B510000000000000000000414E474C453B484FF2
:10B5200052495A4F4E3B4241524F3B4D41473B439C
:10B53000414D535441423B43414D545249473B4195
:10B54000524D3B47505320484F4D453B47505320A9
:10B55000484F4C443B50415353544852553B484547
:10B560004144465245453B4245455045523B4C457A
:10B57000444D41583B4C4C49474854533B48454146
:10B580004441444A3B00524F4C4C3B504954434881
:10B590003B5941573B414C543B506F733B506F7389
:10B5A000523B4E6176523B4C4556454C3B4D4147D4
:10B5B0003B56454C3B00B56206010300F00500FF19
:10B5C00019B56206010300F00300FD15B56206011E
:10B5D0000300F00100FB11B56206010300F000005A
:10B5E000FA0FB56206010300F00200FC13B5620613
:10B5F000010300F00400FE17B5620601030001021A
:10B60000010E47B562060103000103010F49B5624F
:10B6100006010300010601124FB562060103000195
:10B6200012011E67B56206160800030703005108E1
:10B6300000008A41B56206080600C800010001004A
:10B64000DE6A1048494A4B4C4D44454647FF20218D
:10B6500022232425262748494A4B4C4DFF104849B0
:10B660008A8B8C8D84858687FF20212223242526A2
:10B670002748498A8B8C8DFF000C01400800100080
:10B68000000C0140100010000008014000101400E0
:10B69000000000000000F03F000000000000F83F44
:10B6A00000000000000000000000004003B8E23F7E
:10B6B000000000000000000006D0CF43EBFD4C3E30
:10B6C000033333333333E33FFFAB6FDBB66DDB3F25
:10B6D0004D268F515555D53F01411DA96074D13F6D
:10B6E00065DBC9934A86CD3FEF4E454A287ECA3F67
:10B6F0003E5555555555C53F93BDBE166CC166BFE9
:10B700002CDE25AF6A56113FF16BD2C541BDBBBEE1
:10B71000D0A4BE726937663E004040404040404081
:10B720004040414141414140404040404040404014
:10B7300040404040404040404005020202020202B8
:10B740000202020202020202022020202020202007
:10B75000202020020202020202029090909090901B
:10B7600010101010101010101010101010101010D9
:10B77000101010100202020202028888888888884D
:10B780000808080808080808080808080808080839
:10B7900008080808020202024000000019B7000869
:10B7A0000000000000000000000000006E83F9A20D
:10B7B0002915444ED15727FCC0DD34F5999562DB3D
:10B7C0004190433CAB6351FE4D505536303530000F
:10B7D000565441494C34005934004144584C333498
:10B7E000350048455836005936004F43544F5838B5
:10B7F00000414343004641494C53414645004149BD
:10B8000052504C414E45004D41470048454C495F20
:10B8100039305F444547004759524F5F534D4F4FB2
:10B820005448494E47004C45445F52494E470046F4
:10B830004C59494E475F57494E47004249005452C0
:10B84000490047494D42414C00494E464C49474802
:10B85000545F4143435F43414C00435553544F4D64
:10B860000048454C495F3132305F4343504D0050F2
:10B87000504D005350454B5452554D004241524F8C
:10B88000005155414450004D4F544F525F53544F57
:10B8900050004F43544F464C41545000534F4E417B
:10B8A0005200475053005642415400534552564FA0
:10B8B0005F54494C5400484558365800515541444E
:10B8C00058004F43544F464C4154580054454C4542
:10B8D0004D45545259006D69647263006770735F1F
:10B8E000706F73725F64006770735F706F735F6413
:10B8F000006770735F6E61765F640067696D626197
:10B900006C5F70697463685F6D69640067696D621C
:10B91000616C5F726F6C6C5F6D69640077696E67F4
:10B920005F6C6566745F6D69640077696E675F72EE
:10B93000696768745F6D69640079617764656164E3
:10B9400062616E64006D696E636F6D6D616E64003F
:10B95000766261746D696E63656C6C766F6C746130
:10B96000676500766261746D617863656C6C766F93
:10B970006C74616765006D7075363035305F736368
:10B98000616C6500766261747363616C65007472EA
:10B99000695F7961775F6D6964646C650066616990
:10B9A0006C736166655F7468726F74746C65006D4A
:10B9B000696E7468726F74746C65006D6178746818
:10B9C000726F74746C65006C6F6F7074696D650074
:10B9D0006770735F74797065006163635F6861723B
:10B9E0006477617265006665617475726500736580
:10B9F00072766F5F70776D5F72617465006D6F74E2
:10BA00006F725F70776D5F72617465006E61765FF3
:10BA1000736C65775F726174650073657269616CE0
:10BA20005F6261756472617465006770735F626103
:10BA30007564726174650073617665006261726F2E
:10BA40005F7461625F73697A65006261726F5F63E0
:10BA500066006261726F5F6E6F6973655F6C7066BE
:10BA6000006779726F5F6C7066006E61765F636FFE
:10BA70006E74726F6C735F68656164696E67006491
:10BA80005F706974636800695F70697463680070EF
:10BA90005F7069746368006770735F706F73725F63
:10BAA00069006770735F706F735F69006770735FC1
:10BAB0006E61765F69006D696E636865636B006DCA
:10BAC0006178636865636B0070697463685F64695B
:10BAD00072656374696F6E5F6C00726F6C6C5F642B
:10BAE0006972656374696F6E5F6C00616C745F6826
:10BAF0006F6C645F7468726F74746C655F6E65758B
:10BB00007472616C006C697374206F72202D7661A1
:10BB10006C206F722076616C00645F6C6576656C7A
:10BB200000695F6C6576656C00705F6C6576656C4E
:10BB300000645F726F6C6C00695F726F6C6C007098
:10BB40005F726F6C6C0072657461726465645F61D2
:10BB5000726D0067696D62616C5F70697463685FC4
:10BB60006761696E0067696D62616C5F726F6C6CB2
:10BB70005F6761696E006E61765F73706565645FB3
:10BB80006D696E0067696D62616C5F70697463688E
:10BB90005F6D696E0067696D62616C5F726F6C6C7E
:10BBA0005F6D696E0077696E675F6C6566745F6D67
:10BBB000696E0077696E675F72696768745F6D6947
:10BBC0006E007472695F7961775F6D696E0076658A
:10BBD0007273696F6E006D61675F6465636C696E37
:10BBE0006174696F6E007961775F6469726563740F
:10BBF000696F6E006770735F706F73725F7000675C
:10BC000070735F706F735F70006770735F6E6176E3
:10BC10005F70006D61700068656C700070697463BE
:10BC2000685F646972656374696F6E5F7200726FDA
:10BC30006C6C5F646972656374696F6E5F72006DCE
:10BC4000617070696E67206F66207263206368613F
:10BC50006E6E656C206F72646572006465736967EF
:10BC60006E20637573746F6D206D69786572006105
:10BC700063635F6C70665F666163746F720067799F
:10BC8000726F5F636D70665F666163746F7200737D
:10BC900070656B7472756D5F686972657300676952
:10BCA0006D62616C5F666C61677300646566617587
:10BCB0006C7473006770735F77705F72616469752D
:10BCC000730073686F772073797374656D20737474
:10BCD0006174757300736574006578697400645FDE
:10BCE000616C7400695F616C7400705F616C7400FA
:10BCF0007361766520616E64207265626F6F740097
:10BD0000726573657420746F2064656661756C7408
:10BD10007320616E64207265626F6F74006D697864
:10BD20006572206E616D65206F72206C697374009E
:10BD30006E616D653D76616C7565206F7220626C19
:10BD4000616E6B206F72202A20666F72206C69739F
:10BD50007400645F79617700695F79617700705F73
:10BD6000796177004D4D4138343578006E61765FEA
:10BD700073706565645F6D61780067696D62616CA1
:10BD80005F70697463685F6D61780067696D626197
:10BD90006C5F726F6C6C5F6D61780077696E675F66
:10BDA0006C6566745F6D61780077696E675F726954
:10BDB0006768745F6D6178007472695F7961775F3D
:10BDC0006D617800636D6978006661696C736166A6
:10BDD000655F64656C6179006661696C7361666555
:10BDE0005F6F66665F64656C6179006163635F6C59
:10BDF00070665F666F725F76656C6F6369747900F9
:10BE000024504D544B3235312C31393230302A32B6
:10BE1000320D0A0024505542582C34312C312C302C
:10BE20003030332C303030312C31393230302C300E
:10BE30002A32330D0A0024505542582C34312C310B
:10BE40002C303030332C303030312C3338343030EB
:10BE50002C302A32360D0A0024504D544B323531E5
:10BE60002C33383430302A32370D0A0024504D54E8
:10BE70004B3235312C35373630302A32430D0A00FB
:10BE800024505542582C34312C312C303030332C46
:10BE9000303030312C35373630302C302A32440DAA
:10BEA0000A0024505542582C34312C312C3030307B
:10BEB000332C303030312C3131353230302C302A87
:10BEC00031450D0A0024504D544B3235312C31315F
:10BED000353230302A31460D0A000000FCBE000821
:10BEE00000000020D40400007095000840C0000845
:10BEF000D4040020241A00005498000841133EB8CE
:10BF00001B0881041ABC041A3B041A420413E7B745
:10BF10001B08E2041A2F0C1AD7081AB6081AEA08E6
:10BF20001A92081AC2041AFE0C1A61081A0B041A93
:10BF3000D00C1A5A08411A6F081AA6041A49041A92
:10BF400073041A87041AAB041A17041A26041AA2D7
:10BF5000041AF5301A9C085ACC341AF1101A7C0CC9
:10BF60001A0704291829244113FFBD1B08DA1C1ADB
:10BF7000C8041A640C410228200351093DCBDC059A
:10BF80000201A0CBDE0502710211030234018B8095
:10BF90003F04018E338025324B329632E113C201C9
:10BFA0001314BE1B0836041A80041AA204111904C3
:10BFB0001A58041A6C042AC510014BE203124045BA
:10BFC000080140018A1C1032029A041032049A08B7
:10BFD0001029912A0C104A041042408A1D102A8010
:10BFE0000B69104A0C609A081029602A0C103B2C2F
:10BFF00001301129211A1B05691019612A0C104AF8
:10C00000083039602A1E454910396099102940AA24
:10C01000081019611A0C10134EB61B0842041A6955
:10C02000041A5D040144B94584A24A04380C010293
:10C030000304060708090204062329106914C10035
:04000005080000ED02
:00000001FF
